:020000040800F2
:2000000028310020613300087D3300088133000885330008893300088D330008000000000B
:20002000000000000000000000000000913300089533000800000000993300089D33000878
:2000400000F09ABF00F026B800F024B800F022B800F020B800F01EB800F01CB800F01AB8DF
:2000600000F018B800F016B800F014B800F012B800F010B800F0F2BF00F0D8BF00F083BF7A
:2000800000F091BF01F014B801F01CB8A1330008A5330008DFF800F000000000F8B500F07E
:2000A0006BFFDFF85C4A04F50A750146284600F03FFDDFF8506A4FF400520021304600F053
:2000C000E7FF06F200474FF4B0720FF6AC41384600F0E8FF0B222946384600F0E3FF0FF262
:2000E000600518222946304600F0DCFF1822294606F5007000F0D6FFDFF80C0AC6F8160413
:20010000A022DFF8081A06F5C06000F0CBFF50220FF2FC1106F5006000F0C4FF40220FF25E
:20012000402106F5206000F0BDFFA0680021C171017241716068C1604161C1618161F1BD7A
:20014000F8FFFFFFFFFFFF6F0007800009A0000BC000FFFFFFFF0F0070B50D46B5F5805F37
:2001600008D14FF400720146DFF89809BDE8704000F098BFB5F5205F08D14FF40072014698
:20018000DFF88C09BDE8704000F08CBFB5F5804F08D14FF400720146DFF87809BDE8704068
:2001A00000F080BFB5F51A4F3CD3DFF858694FF40072014606F5C06000F074FFDFF840497C
:2001C0004FF40072314604F1280000F06BFFA068017A002926D1C07900280FD1B5F52A4F75
:2001E00004D300F04FFAA168087270BD2088002818D000F047FAA168087270BD012811D19B
:200200002088002807D0B5F51C4F04D300F093FBA168087270BDB5F52C4F03D300F08BFBAC
:20022000A168087270BD10B50446002907D14FF400720FF64411BDE8104000F033BFB1F572
:20024000805F07D14FF40072DFF8B818BDE8104000F028BFB1F5205F07D14FF40072DFF836
:20026000B018BDE8104000F01DBFB1F5804F07D14FF40072DFF89C18BDE8104000F012BFB2
:20028000B1F5004F0CD14FF40072002100F000FFA0220FF644412046BDE8104000F002BF6F
:2002A000B1F5024F0CD14FF40072002100F0F0FE50220FF25C012046BDE8104000F0F2BEEB
:2002C0006FF40240401841F2FF7290420DD24FF400720021204600F0DBFE40220FF28001E3
:2002E0002046BDE8104000F0DDBEB1F51A4F4FF4007206D3DFF820182046BDE8104000F021
:20030000D1BE00212046BDE8104000F0C1BE00007B00380031004200320031003700330070
:2003200033002D0036003800440039002D0034003000350039002D00410035003700330066
:200340002D004500410030004400320033003200450039003300320031007D00000000004E
:200360002E202020202020202020203200478A5A7945794500008A5A794504000000000090
:200380002E2E2020202020202020201000478A5A7945794500008A5A794500000000000088
:2003A0002DE9F84F2024DFF85C672AE0522805D1697A442902D1A97A592921D0552805D19C
:2003C000697A532902D1A97A452919D0452805D1697A522902D1A97A522911D04E2805D132
:2003E000687A4F2802D1A87A542809D04520287252206872A872DFF8080780680321017290
:020000040800F2
:200400002034B4F5007F80F21381A01900F20045002028732878E528F2D00028F0D0E87AF6
:200420002028EDD1287A482836D1697A452933D1A97A582930D1DFF8C876A87EE97E00EB16
:2004400001200005000D38804FF47A7000F03AFEB8680021C171017A002904D002290FD067
:20046000042907D012E052212972442169725921A9720BE04521297252216972A97205E069
:200480004E2129724F2169725421A972E97D491CE97503210172B3E741287BD1697A442918
:2004A00078D1A97A522975D1DFF85476A87EE97E00EB01200005000D38804FF47A7000F0EE
:2004C00001FED7F80880002088F8070088F80800D7F80490C9F800004FF0020A07E098F8B1
:2004E000080040F0040088F808000AF1010ABAF10A0F27DA96F800063028F0D196F801062B
:200500007828ECD10AEB060090F80016A1F13002D2B20A2A08D3A1F14102D2B2062A03D32F
:200520006139C9B20629DAD2D9F800100901C9F800108B4690F8000600F024FA5844C9F845
:200540000000D2E798F8080000281AD1D9F80000DFF8C815884203D300F025FD002806D101
:200560004E2028724F2068725420A8720EE0B8680121C17153202872452068725420A87260
:2005800004E04520287252206872A872B8680321017235E7422830D1697A49292DD1A97A5E
:2005A0004E292AD1DFF85875A87EE97E00EB01200005000D38804FF47A7000F083FDB86805
:2005C000C179002906D14E2129724F2169725421A97205E052212972442169725921A97234
:2005E000C179022901D10021C171C179012901D10221C1710321017202E753287FF4D6AEF4
:20060000697A45297FF4D2AEA97A54297FF4CEAEDFF8EC74B868C17900297FF4F1AE5521C5
:200620002972532169724521A97203210172E7E6BDE8F18F10B5DFF8C844A068007A032871
:200640001ED100F04AFE0028FBD1002000F047FD4FF4C87000F036FD012000F040FD00F04F
:2006600049FEA068002101724171616800224A61CA6011462180C179022901D11146C1716D
:2006800010BD00002DE9F843DFF8744460680021016106E0A0680021417160680169491C0A
:2006A000016166683069B0F5007F80F04181A56869790E29F1D8DFE801F0091221313E5376
:2006C00060768299A7C5D3E0EA00E6E7DFF83414401890F800063A2840F02881D3E0DFF889
:2006E0002414401890F8000600F04CF90001A870002070616879401C6871CEE7AE78DFF8D5
:200700000414401890F8000600F03CF98019A870A878E8706879401C6871BEE7DFF8E41304
:20072000401890F8000600F02DF9000170606879401C6871B1E77768DFF8C813401890F8CD
:20074000000600F01FF9C0197060E87871680818E8707068000270606879401C68719CE7EE
:20076000DFF8A013401890F8000600F00BF9000128716879401C68718FE72F79DFF88413D9
:20078000401890F8000600F0FDF8C01928717068297908187060E87829790818E870687957
:2007A000401C687179E7D749401890F8000600F0E9F8000168706879401C68716DE76E78A4
:2007C000D049401890F8000600F0DCF880196870E87869780818E8706879401C6871A978F5
:2007E00000297FF45AAF801C687156E7C549401890F8000600F0C6F800017169E2688854FF
:020000040800F2
:200800006879401C687148E77769D4F80C8017F80890BC49401890F8000600F0B3F84844A2
:2008200007F80800E878716911F808100818E8707069401C7061A978884224D26879401EB8
:2008400068712AE7EE78AF49401890F8000600F099F806EB0010E8706879401C68711CE777
:20086000EE78A849401890F8000600F08BF88019E870E878002859D105E0A249401890F875
:2008800000060D2852D16879401C687105E79D49401890F800060A2848D10020E871687888
:2008A000042809D1D4F80C8098F8000098F80110090401EB0060B0606878012838D0002807
:2008C0007FF4E8AE7068B168081870609349884201D202202DE00020706103E06068416940
:2008E000891C416160684169A26892789142BFF4D1AE4068081800F01EFD60684169E26897
:200900008B5C406808184D1CA668B678B54204D143F47F4100F0FEFC06E08918497803EBA0
:20092000012189B200F0F6FC0428D7D0042000E00020BDE8F28338B50024714D00E0A41CF8
:20094000B4F5007F1CD268680168C068401800F0F2FC68686B49611891F8002691F801169E
:2009600002EB012189B20268C068801800F0D2FC6968CA68921CCA600428E0D0042032BD7B
:20098000002032BD10B585B0044600A80FF2D411112200F0F5FCA4F16100C0B21A2800D2E6
:2009A000203C002000E0401CC0B2102805D200A9415CE4B2A142F6D100E0002005B010BDF6
:2009C00038B54F4CA2681378002B05D1400260614802A061012010701078012833D12569C7
:2009E0006068806900280FD161692846FFF71BFC40229821284600F0EEFC60684FF4E0713A
:200A000081614020E0610CE040229821E069401900F0E1FC6068816940398161E069403017
:200A2000E0614021012000F09FFD3021012000F00BFD606940306061A0694038A061384801
:200A4000816840398160A06900280BD16068002181610846E0616061324803210170A06814
:200A60000021017031BD70B5254C6268D3694033A5682E78002E05D1400220624802606260
:200A8000012028702878012827D1002007E02569254E865D4E55401CD169491CD161D169E7
:200AA0009942F4D3214D2888216A41182162636A181A6062C00506D10020D061A1F500715A
:200AC0002069FFF749FB164881682A88891A81604FF44051022000F0CBFC606A002803D064
:200AE00010480078042809D160680021C1610121002000F0B7FEA0680021017070BD000067
:200B0000000000201C040020188DDD40D80E00081C0600201C0800201C0A002000400008B1
:200B2000EC2C0020B82C0020582C0020BA2C002010B41C2203E0303300F8013B121F1346C9
:200B40005BB2002B0AD421FA02F303F00F031C460A2CF0DB373300F8013BEFE70021017001
:200B600010BC70473031323334353637383941424344454600000000EB3C904D53444F5313
:200B8000352E3000020108000200020010F80C00010001000000000000000000000029A2D2
:200BA00098E46C4E4F204E414D4520202020464154313220202033C98ED1BCF07B8ED9B8B0
:200BC00000208EC0FCBD007C384E247D248BC199E83C01721C83EB3A66A11C7C26663B077A
:200BE000268A57FC750680CA0288560280C31073EB33C98A461098F7661603461C13561EC7
:020000040800F2
:200C000003460E13D18B7611608946FC8956FEB82000F7E68B5E0B03C348F7F30146FC118A
:200C20004EFE61BF0000E8E600723926382D741760B10BBEA17DF3A66174324E740983C70C
:200C4000203BFB72E6EBDCA0FB7DB47D8BF0AC9840740C487413B40EBB0700CD10EBEFA0AD
:200C6000FD7DEBE6A0FC7DEBE1CD16CD19268B551A52B001BB0000E83B0072E85B8A5624C1
:200C8000BE0B7C8BFCC746F03D7DC746F4297D8CD9894EF2894EF6C606967DCBEA03000098
:200CA000200FB6C8668B46F86603461C668BD066C1EA10EB5E0FB6C84A4A8A460D32E4F757
:200CC000E20346FC1356FEEB4A525006536A016A10918B4618969233D2F7F691F7F6428796
:200CE000CAF7761A8AF28AE8C0CC020ACCB80102807E020E7504B4428BF48A5624CD136155
:200D000061720B40750142035E0B497506F8C341BB000060666A00EBB04E544C4452202087
:200D2000202020200D0A52656D6F7665206469736B73206F72206F74686572206D6564696E
:200D4000612EFF0D0A4469736B206572726F72FF0D0A507265737320616E79206B65792005
:200D6000746F20726573746172740D0A00000000000000ACCBD855AA4446552056335F34EB
:200D8000325F4408000000000000000000008A5A794500000000000042200049006E006655
:200DA000006F000F007272006D006100740069006F0000006E000000015300790073007495
:200DC0000065000F00726D00200056006F006C00750000006D00650053595354454D7E3194
:200DE00020202016005E63705D455D45000064705D45020000000000412E005F002E005440
:200E00000072000F007F6100730068006500730000000000FFFFFFFF7E3120202020202053
:200E200054524122004A8A5A7945794500008A5A7945050000100000E552415348457E3141
:200E400045464D1200478A5A7945794500008A5A7945040000000000412E005400720061C5
:200E60000073000F00256800650073000000FFFFFFFF0000FFFFFFFF5452415348457E311D
:200E80002020201200478A5A7945794500008A5A7945040000000000412E006600730065E6
:200EA0000076000F00DA65006E0074007300640000000000FFFFFFFF46534556454E7E3143
:200EC00020202012004D8A5A7945794500008A5A79450D00000000002E2020202020202036
:200EE00020202010005E63705D455D45000064705D450200000000002E2E20202020202079
:200F000020202010005E63705D455D45000064705D450000000000004247007500690064AB
:200F20000000000F00FFFFFFFFFFFFFFFFFFFFFFFFFF0000FFFFFFFF0149006E0064006532
:200F40000078000F00FF6500720056006F006C00750000006D006500494E444558457E3150
:200F600020202020007263705D455D45000064705D4503004C00000041480168426851189E
:200F800080684018704710B50446FFF7F5FF0A233C4A01463C4800F017F8844201D101202B
:200FA00010BD002010BD10B5FFF7E6FF37490C680A23344A0146344800F006F8844201D1EF
:200FC000012010BD002010BDF0B403F11506C3F14304C3F151050A330FE0C0EB40104FEA1E
:200FE000670C07EB9C7C4FEAAC0CA7EB8C07FF0021FA07F7FFB238185B1C1BB21F46B742A3
:020000040800F2
:20100000EBDB0DE0C0EB40104B1001EB93739B10A1EB8301C90022FA01F1C9B20818641C28
:2010200024B22146A942EDDBF0BC704770B504460D461646FFF7B7FF002801D1002070BD4C
:20104000FFF79AFF0023324601462046FFF7BCFF854201D1012070BD002070BD70B5044665
:201060000D461646FFF79FFF002801D1002070BD0023324629462046BDE87040A4E7000096
:20108000E8F7FF1F011020D502DEC0DEFC3F000810B5044610460A460146204600F03EFC00
:2010A000204610BD10B5044600F05AF9204610BD0FF27C11082802D201EB0010704701F141
:2010C0008000704700214FF6FF7302E04F4A1360491C40F2DC5242439142F7D370474C49E0
:2010E0004FF400620A614FF480520A61002808680BD120F4404040F440500860086820F4A8
:20110000402040F440300860704720F4804040F430400860086820F4802040F430200860BC
:201120007047000080F308887047704710B500F029FC4FF4803000F03DFC00F055FC102020
:2011400000F0BCFC022000F0AFFC324C6068324908436060206840F080702060012000F025
:201160005CFC012000F05CFC392000F076FC0028FAD0022000F057FC00F05CFC0828FBD158
:201180001420606140F60D20A0614FF42000E0610120BDE8104000F052BC80B501464FF083
:2011A000006000F05DFD4FF4C06000F013FD14208DF8000001208DF801008DF802008DF8B6
:2011C000030000A800F00BFD13208DF8000001208DF8010000208DF8020001208DF80300BD
:2011E00000A800F0FCFC01BD0C484FF6FF71C1600B4901600B4941600B484FF6FE71C160A5
:201200000A4901604FF08831416070470C10014004080140001002400A846800000801408F
:201220008888880883B8BB8B000C014003888344312E33300000000000000000000000002C
:2012400053544D3332463130335438000000000056474D393631360000000000000000000F
:201260004D4355277320414443000000000000004E6F6E6500000000000000000000000077
:2012800056332E3432410000000000000000000030000000000000000000000000000000C0
:2012A0005669727475616C204D534400000000002D2D2D2D2D2D0000000000000000000035
:2012C0000A48012101600021016041604FF4E051074A1180016000207047044801210160B9
:2012E000002141600321016000207047405C0040222D00200448C0610221017203490162D3
:20130000034A426208680047C42C00200C0300206403002038B504460D46104800F03AFC57
:20132000052802D0342000F014FC29462046BDE8344000F0F5BB10B50446A0050CD10748EC
:2013400000F028FC052802D0342000F002FC2046BDE8104000F0C5BB10BD0000A086010079
:2013600062B38B0708D0521E11F8013B00F8013B00F024808B07F6D1830740F0208000BFFF
:20138000103A07D330B4B1E83810103AA0E83810F9D230BC530724BFB1E80810A0E8081005
:2013A00044BF51F8043B40F8043BD20724BF31F8022B20F8022B44BF0B7803707047083AE2
:2013C00007D3B1E80810083A40F8043B40F804CBF7D25307E4E710B4490001F1804101F51E
:2013E000C041521C521009E010F8013B10F8014B43EA042321F8023B891C521EF4D110BC4B
:020000040800F2
:201400007047490001F1804101F5C041521C521004E051F8043B20F8023B521EF9D17047A0
:201420004FF6F8710840DFF8A4110860704710B4DFF89C2152F8203048F68F142340194379
:2014400042F8201010BC704710B4DFF8842152F8203048F6BF742340CC0601D583F01003C3
:20146000890601D583F0200342F8203010BC704710B4DFF85C2152F820304BF68F7423400B
:20148000CC0401D583F48053890401D583F4005342F8203010BC7047DFF8341151F820207D
:2014A0004BF68F731A4082F4405241F820207047DFF81C1151F8202048F68F631A4041F807
:2014C00020207047DFF8081151F82020520409D551F8202092B248F68F731A4042F4804209
:2014E00041F820207047DFF8E81051F82020520609D551F8202092B248F68F731A4042F095
:20150000400241F820207047DFF8C020126892B202EBC000DFF8BC204908490042F8101090
:201520007047DFF8A820126892B202EBC000DFF8A8204908490042F810107047DFF88C102D
:20154000096889B201EBC000DFF8881051F8100080B270471D49096889B201EBC0001E495D
:2015600051F8100080B27047184A126892B202EBC0001A4A42F810107047144A126892B2CB
:2015800002EBC000164A02EB40003F290AD34A091F23194200D1521E92B2910241F400414E
:2015A000016070474A08C90700D5521C92B29102016070470549096889B201EBC0000849C8
:2015C00051F810008005800D70470000505C0040005C004000600040086000400460004075
:2015E0000C6000400146C9B2090241EA1020704780B5AC4890F8201002290FD022D3042953
:2016000002D014D305291DD1002180F820104FF440510220BDE80440FFF72ABFC17B2829E1
:2016200010D1816A406ABDE8044000F073BB0121002000F017F94FF440510220BDE804400C
:20164000FFF716BF01BD38B5964CE57B0220FFF7B1FF60840246D8219348FFF7D2FE94F8B8
:201660002000002802D0012803D016E0BDE831401FE02A2D05D1A16A606ABDE8344000F03E
:2016800078BB012000F01AF92421052000F03AFB00210220BDE83440E4E0022000F00EF92B
:2016A0002421052000F02EFB00210220BDE83440D8E010B500207B4C03E07B49415C01554D
:2016C000401C618C8842F8D3784862684260A26882601F290DD0022000F0F0F80020206055
:2016E0001A21052000F00EFB00210120BDE81040B8E0E07B282801D02A280FD1617CA27C19
:20170000120442EA0161E27C41EA0221227D11436162A17DE27D42EA0121A1622168644ABE
:2017200091427AD163490968627B914204D3A17B491EC9B210290BD3022000F0BFF82421C4
:20174000052000F0DFFA00210120BDE8104089E000284AD003282CD008285AD00A2858D0DE
:2017600012282AD0152854D01A282ED01B2828D01D284ED01E2824D023282ED0252830D026
:20178000282836D02A283AD02F283ED0552840D05A281ED088283CD08A283AD08F2838D0FE
:2017A0009E2836D0A82834D0AA2832D0AF2830D033E0BDE8104000F09DBABDE8104000F0AA
:2017C00063BABDE8104000F0A1BABDE8104000F089BABDE8104000F089BABDE8104000F077
:2017E00062BABDE8104000F06DBABDE8104000F008BBA16A606ABDE8104000F08BBAA16A0F
:020000040800F2
:20180000606ABDE8104000F0B4BABDE8104000F0DDBABDE8104000F0F8BA022000F04EF840
:201820002021052000F06EFA00210120BDE8104018E010B50C4622469821FFF7CCFD21465D
:201840000120FFF791FE30210120FFF7FDFD1548032180F8201015488168091B81600021EB
:20186000017310BD10B50C46104B1349196018730D2298211846FFF7AEFD0D210120FFF729
:2018800073FE0848052180F82010002C08D0042180F8201030210120BDE81040FFF7D4BDFA
:2018A00010BD0000982C0020582C0020EC2C002055534243102D00205553425380B5002877
:2018C00003D002280ED006D301BD10210120BDE80440FFF7B9BD4FF480510220BDE80440D0
:2018E000FFF7C6BD10210120FFF7AEFD4FF480510220BDE80440FFF7BBBD50F8041B61B176
:2019000050F8042BD30744BFA9F101039A18002342F8043B091FFAD1EFE7704762F30F2281
:2019200062F31F42401810F0030308D0C91A1FD3DB0748BF00F8012D28BF20F8022D130096
:2019400030B414461546103928BF20E93C00FAD8490728BF20E90C0048BF40F8042D890062
:2019600028BF20F8022D48BF00F8012D30BC7047C91818BF00F8012DCB0728BF00F8012DAC
:20198000704700004048016841F00101016041683E4A1140416001683D4A114001600168DD
:2019A00021F480210160416821F4FE01416000218160704734490A6822F480320A600A6866
:2019C00022F480220A60B0F5803F03D0B0F5802F05D07047086840F48030086070470868EB
:2019E00040F4A0200860704710B582B0002000900446312000F031F80099491C00910028C2
:201A000003D10098B0F5A06FF3D1312000F025F8002800D00124204616BD1E4908607047A8
:201A20001E49086070471C490A68920850EA8200086070471848006800F00C0070471849F8
:201A400008607047174A0029116802D008431060704721EA000010607047002142090A4B2D
:201A6000012A01D11A6804E0022A01D11A6A00E05A6A012300F01F0003FA00F0024200D0A9
:201A80001946084670470000001002400000FFF8FFFFF6FE000042420410024060004242E9
:201AA000D800424218100240DFF8D0100A6802F038020A600A68104308607047DFF8BC101A
:201AC0000A6822F010020A600A68104308607047DFF8AC00DFF8AC100160DFF8AC100160B7
:201AE000704770B5054640F6FF76304600F052F8042814D1DFF89440206840F0020020606E
:201B00006560206840F040002060304600F042F8012804D0216841F6FD721140216070BDBD
:201B200070B504460D460F2000F034F804280FD1164E306840F00100306025800F2000F00B
:201B400029F8012804D0316841F6FE721140316070BD0F490860704704200D490A68D207DC
:201B600001D5012070470A68520701D5022070470968C90600D503207047000000200240EC
:201B80000420024023016745AB89EFCD102002400C20024010B50446FFF7DEFF04E000F089
:201BA0000BF8FFF7D9FF641E012801D1002CF6D1002C00D1052010BD81B000200090FF20F5
:201BC000009002E00098401E009000980028F9D101B07047274908432749086070472DE9BB
:201BE000F04105782B460121C278002A2FD0224A126802F4E062C2F5E062120A23F00303F5
:020000040800F2
:201C00001B4C1F5905F00305ED00FF26AE40B74390F801C0C2F1040E0CFA0EFC90F802E066
:201C20004FF00F0828FA02F202EA0E0242EA0C021201AA4032403A431A51007842110F4B86
:201C400000F01F0001FA00F043F8220006E05811064A05F01F03994042F82010BDE8F0811E
:201C6000074A1140084307490860704780E100E000E400E00000FA050CED00E000E100E06A
:201C800080FFFF1F08ED00E08749087CC00702D58648052105E00FF23020C97C252900D350
:201CA0002421FFF7C6BD824800218180022181710021C1714172022181720021C1720C21C8
:201CC000FFF7B7BD7B48002101800F218170FF21C17000218180022181710021C171082110
:201CE000FFF7A7BD04217448FFF7A3BD08217348FFF79FBD6C48C17C132900D31221704832
:201D0000FFF797BD6E4A90701173704701210020FFF7A8BD70B504460D466A4E307800289F
:201D20001FD12A462146282000F08CF800281FD05D48007B000607D5022030702946204670
:201D4000BDE87040FEF73CBE0220FFF7B7FD24210520FFF7D7FF01210846BDE87040FFF782
:201D600081BD022804D12046BDE87040FEF728BE70BD10B5534C2278002A20D10A460146B3
:201D80002A2000F05FF800281FD04748007B000608D4012020704FF440510220BDE8104013
:201DA000FFF766BB0020FFF789FD24210520FFF7A9FF00210120BDE81040FFF753BD012A00
:201DC00003D1BDE81040FEF74EBE10BD80B536488168002908D1007C400705D401210020F0
:201DE000BDE80440FFF73EBD0220FFF767FD24210520FFF787FF00210120BDE80440FFF786
:201E000031BD01210020FFF72DBD80B526488168002903D10020FFF751FD09E0007B00065B
:201E200003D50020FFF74AFD02E00220FFF746FD20210520FFF766FF00210120BDE8044044
:201E4000FFF710BD80B55118B1F5805F11D92A2802D10220FFF732FD0020FFF72FFD2121C2
:201E60000520FFF74FFF00210120FFF7FBFC002002BD0D498968B1EB422F12D02A2803D18F
:201E80000220FFF71BFD02E00020FFF717FD24210520FFF737FF00210120FFF7E3FC002039
:201EA00002BD012002BD0000982C0020FC2C0020F0030020042D0020180400200C04002087
:201EC000DC030020B82C002000800202200000005669727475616C20444655204469736BCA
:201EE00000000000000000000000000010B5DFF8C047002804D1206801210182002010BD28
:201F0000DFF8B00700680068804720680A3010BD80B5DFF89C070068C178DFF89C27527859
:201F20008A420DD38278002A0AD18288002A07D18172DFF88007006840688047002002BDE3
:201F4000022002BD10B5DFF86847002804D1206801210182002010BDDFF8580700688068B8
:201F6000804720680C3010BD10B5DFF844472068C1784079DFF84427126892699047216851
:201F80008A7A002A14D0002812D1087900280FD1887800280CD1DFF81C070068C068804745
:201FA00020684179C1722068C1780173002010BD022010BD10B5DFF8F8160968002803D184
:201FC00002200882002010BDDFF8F4460020208008787F22104218D1487A0146890603D5CB
:201FE000002141F0020121702178400609D541F001002070DFF8BC060068006980472046E5
:020000040800F2
:2020000010BD01F0FE002070F4E700F07F02012A01D1204610BD00F07F0002281BD14879B2
:2020200000F00F01DFF89C26000652F8210008D500F030001028DDD1002040F001002070D2
:20204000D8E700F44050B0F5805FD3D1002040F001002070CEE7002010BD70B5DFF8500640
:202060000068017811F07F0105D1417A01F0DF014172002070BD022954D14188002951D138
:20208000017900294ED1417921F08005DFF834460A0654F8252002D502F0300201E002F46A
:2020A0004052DFF814361B789D423BD2002A39D0807A002836D0080654F825000BD500F044
:2020C0003000102827D12846FFF70DFA30212846FFF7BAF91FE000F44050B0F5805F1AD1DB
:2020E0004BF68F76002D0CD1DFF8DC0590F82C100020FFF742FA2068304080F44050206046
:2021000009E02846FFF7DEF954F82500304080F4405044F82500DFF89C0500684069804705
:20212000002070BD022070BD38B5DFF884050268537923F08000DFF88C151C0651F82040AA
:2021400002D504F0300401E004F44054DFF868552D78A84207D25588002D04D1002C02D03A
:20216000927A002A01D1022032BD1A0651F8202007D548F6BF731A4082F0100241F82020FA
:2021800006E04BF68F731A4082F4805241F82020DFF82005006880698047002032BD80B5A3
:2021A000DFF80C050068417A41F020014172DFF804050068C0698047002002BDDFF8F0240D
:2021C0001268538A002804D18888C01A108200207047086818187047F8B5DFF8D4442068DD
:2021E00000F110052E88A968080016D0002E14D0A888864200D906463046884707462888B3
:20220000801B28806888301868800020FFF7A2F9324601463846FFF7F4F8288800280CD0D7
:20222000DFF8A8044FF44051018000210846FFF79BF9DFF89C04302101802888A9888842D9
:2022400003D3206803210172F1BD002803D0206805210172F1BD0FD1206806210172DFF838
:202260007404006880B2DFF87014002241F81020DFF85C0430210180F1BD2DE9F041DFF891
:202280003044206800F110052F88002F08D1007A042805D10726DFF838041021018027E008
:2022A000A888B84201D3042600E00226874200D907463846A968884780460020FFF73EF98E
:2022C0003A4601464046FFF786F839460020FFF74BF92888C01B2880688838186880DFF832
:2022E000F00330210180DFF8E4034FF44051018020680672BDE8F08138B50220DFF8B04317
:2023000021684D780A787F231A4230D1092D02D1FFF7FEFD3FE0052D0FD1C878802808D201
:202320008878002805D18888002802D1887A002801D008204AE000202DE0032D0BD1CA78CC
:20234000012A28D18A88002A25D1497A890622D5FFF725FF1FE0012D1DD1CA78012A1AD151
:202360008A88002A17D1497A89060DD413E002F07F01012904D10B2D0DD1FFF7F5FD0AE0BA
:20238000022908D1012D02D1FFF767FE03E0032D01D1FFF7C9FE002809D02846DFF81C13C6
:2023A000096849698847032801D109200EE0002801D008200AE00620C649096889B2C64A1B
:2023C000002342F81130C24930220A802168087231BD38B5B64C206841780025062916D11C
:2023E00001787F22114279D18078012803D1B3480068C56972E0022803D1B0480068056A81
:020000040800F2
:202400006CE003286AD1AD480068456A66E0002940D14288002A3DD1C288022A3AD1027980
:20242000002A37D101787F22114204D18288002A01D1AA4D52E001F07F02012A0DD129460F
:2024400040799E4A126892699047002846D12068807A002842D0A14D40E001F07F010229EA
:202460003CD1407900F00F0100F07002954B000653F8210002D500F0300001E000F4405086
:202480008D4B1B78994229D2002A27D1002825D0924D23E0082905D100787F2108421DD183
:2024A0008F4D1BE00A2919D1017801F07F01012914D1817A002911D0418800290ED10179DF
:2024C00000290BD1C188012908D1294640797B4A126892699047002800D1824D20682900F9
:2024E00007D000214182206885610846A847002006E040787149096809698847032805D04C
:2025000021680A8A4FF6FF739A4203D120680921017231BD022801D0002A02D1082008728A
:2025200031BD087800060CD5C888904200D2088220686249096891F82C108182BDE8314046
:202540009BE60320087261484FF44051018031BD38B56048006880B2634931F8100040001D
:2025600000F1804505F5C045514C2068017A092917D015F8011B0170206815F8011B4170F1
:20258000AD1C35F8020BFFF72DF821684880AD1C35F8020BFFF726F82168888020686988AB
:2025A000C1802068012101722068C088002802D1FFF7A2FE01E0FFF70CFFBDE8314042E042
:2025C00010B53B4C2068017A022901D0042904D1FFF753FE2068007A16E0062913D14178A3
:2025E00005290AD101787F22114206D1C07800F044F830480068006A804730480068806851
:202600008047082000E0082021680872BDE8104019E010B5264C2068007A032801D0052870
:2026200004D1FFF7D9FD2068007A08E0072805D122480068C0688047082000E00820216890
:202640000872BDE8104080B51F4890F82C100020FEF793FF16480068017A082906D11B4957
:202660004FF480520A801A4910220A80007A092801D1012002BD002002BD70B40E49097864
:202680000022104C48F68F7609E01346DBB254F82350ADB235401D4344F82350521C8A42CE
:2026A000F3D340F080001149086070BC70470000E02C0020E82C002014040020E42C002037
:2026C000182D0020005C00400C0300201C2D00201E2D0020505C004004600040B51F00088A
:2026E000ED1E0008451F0008086000404C5C004070470000F8B58478303CE4B20A2C00D261
:202700002246C478303CE4B20A2C00D2234600783038C0B20A2800D20146002413E02018B6
:202720000FF2C415182606FB01477F5D80F8607006FB02477F5D80F8907006FB0346755D5A
:2027400080F8A850641C5548182CE8DB002409E00C220146204600EB40039800C0B200F0D5
:2027600004F8641C082CF3DBF1BD70B50C46154600F1200600213046C0B200F054F86D1C76
:2027800021462846C0B200F03DF8044601213046C0B200F048F821462846C0B2BDE87040AD
:2027A00030E04049086040483C2202700968C9B23B4800F0D1B910B58CB000A80FF2F0013C
:2027C0003022FEF7DDFD0020354903E000AA825C4254401C2E28F9DB344C4FF48071204699
:2027E00000F02BFA0220FEF76DFC4FF48071204600F021FA0220FEF765FC2E20FFF7D1FF13
:020000040800F2
:202800000CB010BD10B50C46254940220A70012203E014F8013B5354521C8242F9DBFFF7DD
:20282000C0FF204610BD30B583B000AA0FF2B00330CB30C28DF80500012902D1B1208DF866
:2028400001000020164903E000AA825C4254401C0828F9DB0820FFF7A4FF37BD10B50021FC
:202860002020FFF7E0FF0E4C402020707F220021601CFEF70DFC8020FFF793FF0121202033
:20288000FFF7D1FF402020707F220021601CFEF7FFFB8020BDE8104083E700003402002000
:2028A0001C2400200C2D0020242D00200008014080AE80D5805280A8800F80C080D3800086
:2028C000804080A0808D801480DA8002808180E080D980F180DB803080A480A680AF0000EC
:2028E00080B080218020807F00E010080810E00000000000000F102020100F0000000000FA
:20290000001010F800000000000000000020203F2020000000000000007008080888700060
:20292000000000000030282422213000000000000030088888483000000000000018202090
:2029400020110E00000000000000C02010F800000000000000070424243F2400000000009A
:2029600000F8088888080800000000000019212020110E000000000000E010888818000086
:2029800000000000000F112020110E000000000000380808C8380800000000000000003F29
:2029A0000000000000000000007088080888700000000000001C222121221C000000000059
:2029C00000E010080810E000000000000000312222110F0000000000000000000000000072
:2029E00000000000003030000000000000000000022000E0401EFDD1704738B504460D4608
:202A0000012D03D12146534800F015F9002D05D121465048BDE8344000F00FB931BD80B5BE
:202A200001210820FFF70EF8C020ADF8000014208DF8030003208DF8020000A9454800F03F
:202A4000A3F800214020FFF7D8FF01218020FFF7D4FF01214020FFF7D0FF0520FFF7C8FFD9
:202A600000218020FFF7C9FF0520FFF7C1FF00214020FFF7C2FF01BD80B500214020FFF75A
:202A8000BCFF00218020FFF7B8FF0520FFF7B0FF01214020FFF7B1FF0520FFF7A9FF012136
:202AA0008020FFF7AAFF0520FFF7A2FF00214020FFF7A3FF0520BDE8024099E738B504463F
:202AC00008250EE000218020FFF797FF0520FFF78FFF01214020FFF790FF0520FFF788FF3C
:202AE00064002846451EC0B200280AD000214020FFF783FF2006E5D501218020FFF77DFF20
:202B0000E4E700214020FFF778FF01218020FFF774FFFF2400E0641EE4B2002C18D005207D
:202B2000FFF766FF80210B4800F07EF80028F2D101214020FFF761FF0520FFF759FF002189
:202B40004020FFF75AFF0520FFF752FF012032BD002032BD000C014070B504460D461646D0
:202B6000FFF75DFF7000C0B2FFF7A8FF03E014F8010BFFF7A3FF2846451EC0B20028F6D1BF
:202B8000BDE8704078E70000F0B40023CC7804F00F02E40601D58C7822430C88E4B2002CF2
:202BA0001CD0046803E0482D00D106615B1C082B13D2012505FA03F635460F882F40AF420E
:202BC000F4D19D000F27AF40BC4302FA05F52C43CD78282DE7D14661E8E704600B88B3F5A3
:202BE000807F1FD34468002319E0012503F1080605FA06F635460F882F40AF420ED19D000B
:020000040800F2
:202C00000F27AF40BC4302FA05F52C43CD78282D00D14661CD78482D00D106615B1C082B7D
:202C2000E3D34460F0BC704700228068084200D00122104670470161704741617047000011
:202C400080B500F007F99348006800218172FEF737FB9148002141604FF404418F4A118044
:202C600001608F480021016001BD10B58D4800218172884800688C49C97941720020FEF717
:202C8000CFFB4FF400710020FEF7D1FB20210020FEF7DAFB18210020FEF743FC834C94F8C2
:202CA0002C100020FEF769FC58210020FEF72CFC0020FEF7FDFB0020FEF7EEFB002101205B
:202CC000FEF7B5FB98210120FEF71EFC20210120FEF7BAFB00210120FEF7CAFB002102201B
:202CE000FEF7A5FBD8210220FEF71BFC94F82C100220FEF742FC4FF440510220FEF7B8FB5D
:202D000000210220FEF7A0FB94F82C100020FEF734FC0020FEF7C0FB0020FFF7AEFC60489B
:202D20000121016062486349016063480021017010BD58480068807A002800D1704780B568
:202D40005748052101600120FEF7CDFB0220FEF7B9FB59480021017001BD55480068554910
:202D6000884202D00220FEF7A9BD70474C480421016070477047704780B546490A68137883
:202D800003F07F03212B10D1FE280ED1508800280BD19088002808D1D088012805D10FF23F
:202DA000A100030003D1022002BD022002BD9061086800214182084600F042F8002002BD3D
:202DC00080B5344909680A7802F07F02212A18D1FF2816D14888002813D18888002810D1A4
:202DE000C88800280DD10120FEF77DFB0220FEF769FB2F482F4901602F48002101700846CD
:202E000002BD022002BD002901D002207047002801D002207047002070472849FFF7CEB9A8
:202E20002749FFF7CBB91B490968C978062901DB00207047234A02EBC101FFF7BFB9000026
:202E4000002805D11348006801210182002070471D4870471D48016842688068002900D1BF
:202E6000704710B41A4B99700C0A1C710C0C9C71090E19729A72110A1973110C9973110E04
:202E800019749874010A1975010C9975000E187610BC7047E02C0020405C0040222D00204F
:202EA000142D0020C42C0020703100080C030020982C002055534243B82C0020FC03002095
:202EC000040400203C030020102D0020E8F7FF1F880300202DE9F0416F4C48F6BF764BF6B0
:202EE0008F7721E05FEA084006D5206840F68F7108402060FFF78DFB206838402988CA04DC
:202F000001D580F48050890401D580F400502060206830406988CA0601D580F01000890652
:202F200001D580F020002060616C5C480180090478D547F6FF716164018811F00F01584DAE
:202F4000297046D1574D216801F440512980216801F0300169802168394081F40051216088
:202F60002168314081F0200121600088C00616D4206880B248F60F7108402060FFF720FBBB
:202F8000D4F800801FFA88F818F4084FB4D0206840F68F7108402060FFF7DAFAACE7D4F8B6
:202FA00000801FFA88F85FEA086007D5206880B248F60F7108402060FFF702FB5FEA085097
:202FC00090D5206840F68F7108402060FFF7C0FA92E754F821801FFA88F85FEA08400DD5E4
:202FE00054F8210040F68F72104044F8210028782D4901EB800050F8040C80475FEA08602E
:020000040800F2
:2030000092D5287854F8201089B248F60F72114044F820102878254901EB800050F8040CA4
:20302000804781E7BDE8F08170B51D4C1A4D2BE047F6FF720260088800F00F00207055F8CF
:203040002060B6B231040DD555F8201040F68F72114045F820102078134901EB800050F857
:20306000040C804730060FD5207855F8201089B248F60F72114045F8201020780B4901EBBA
:20308000800050F8040C80470948026803490A801204CDD470BD0000005C0040202D002013
:2030A000252D00201C2D0020C0030020A4030020445C00402DE9F04500F10801026801EB10
:2030C0008202406800F001034008400002EB80000025AA460024A0460126374602E000270F
:2030E000F44511D1824201D1BDE8F08552F804CB03B1CC4452F804EBE644F1E70D686D18F3
:20310000091D51F804ABAA445545F7D066B115F9014B0026012705E00D686D18091D51F835
:2031200004ABAA445545F7D0002C12D50FB115F8018BF445D3D00CF8018B641CF9D40AE082
:20314000F44518BF5545CBD015F8018B0CF8018B641E002CF4D50126C2E7000012010002A5
:203160000000004083042057000201020301000009022000010100C03209040000020806CC
:2031800050040705810240000007050202400000040309042603530054004D0069006300BF
:2031A00072006F0065006C0065006300740072006F006E0069006300730000002603530017
:2031C00054004D003300320020004D006100730073002000530074006F00720061006700A5
:2031E0006500000010035300540020004D00610073007300FDF79AFFFDF7F6FF1A480068BC
:2032000080050ED5FDF7CFFE18480168184A1140B1F1005F04D144680068FDF783FFA047C2
:20322000FEE70A20FDF74EFF0020FDF758FFC820FDF748FF0120FDF752FF0020FDF7ADFF8A
:20324000FEF758F8FCF72AFFFFF7B5FAFFF706FB0FF22000FFF74EFAFEF73AFCFDF7A0F85B
:20326000FDF7E8F9F8E7000008080140004000080000FF2F332E34330000000070B50D4C8D
:203280000D4D286820800D4E208831880840400505D50B48406880474FF6FF30286020881B
:2032A00031880840000403D5BDE87040FFF712BE70BD0000202D0020445C0040222D00202D
:2032C0000C030020FEF794B9FEF7BDB910B5074979441831064C7C44163404E0081D0A6820
:2032E000511888470146A142F8D110BD080000003000000007E6FFFF0C2900001C0400203E
:2033000000000000B1FDFFFF02000000020000009800000096010000000000201C0400008E
:2033200000F009F8002801D0FFF7D0FF0020FFF761FF00F002F80120704700F001B80000FD
:203340000746384600F002F8FBE70000C046C046024A11001820ABBEFBE700BF2600020003
:2033600001488047014800472D11000871330008C046C046C046C046FFF7D2FFFFF7FEBF29
:20338000FFF7FEBFFFF7FEBFFFF7FEBFFFF7FEBFFFF7FEBFFFF7FEBFFFF7FEBFFFF7FEBF95
:2033A000FFF742BEFFF76ABFFC000F1C2C00203C2C0020452C00201C2A0020810081008183
:2033C000008100DC000104FCFC04070C0810E00000407FFC40076020180F000004FCFB845C
:2033E00007E40C100000407F40FC000003FC000204FC04FB000604FC0400001F20FB400146
:020000040800F2
:20340000201FFA00016060F600016060F9000078FB04018878FC0007605048444241407018
:20342000F000016060F60002E01808FD04020818E0FD00020F3020FD400220300FFB0002E7
:203440000808FCF7000240407FFD40E50027412C00086B2C0008752D0008772D0008792D0F
:203460000008C12D0008072E00081B2E0008212E0008272E0008FC000040FD00049031000E
:203480000804FD00049431000826FD0004BC31000826FD0004880300201AFD0004E4310034
:2034A0000810FD0032F1260008332D0008F1260008F1260008F12600085B2D0008F126003A
:2034C00008F12600086D2D00081A03530054004D0033003200310030F30038C5320008F131
:2034E000260008F1260008F1260008F1260008F1260008F1260008F1260008C9320008F1F0
:20350000260008F1260008F1260008F1260008F126000870FA00000AF1000008FC00000296
:20352000FD00045C31000812FD00047031000820FC000006FA00040301000003FD00000015
:20354000FFFFFFFFFFFFFFFFFFFFFFFFFFFFFFFFFFFFFFFFFFFFFFFFFFFFFFFFFFFFFFFF8B
:20356000FFFFFFFFFFFFFFFFFFFFFFFFFFFFFFFFFFFFFFFFFFFFFFFFFFFFFFFFFFFFFFFF6B
:20358000FFFFFFFFFFFFFFFFFFFFFFFFFFFFFFFFFFFFFFFFFFFFFFFFFFFFFFFFFFFFFFFF4B
:2035A000FFFFFFFFFFFFFFFFFFFFFFFFFFFFFFFFFFFFFFFFFFFFFFFFFFFFFFFFFFFFFFFF2B
:020000040800F2
:020000040800F2
:2040000098350020E1BA000881BA000883BA000885BA000887BA000889BA000800000000AD
:204020000000000000000000000000008BBA00088DBA0008000000008FBA000891BA000840
:2040400021BB000825BB000829BB00082DBB000831BB000835BB000839BB00083DBB0008D0
:2040600041BB000845BB000849BB00084DBB000851BB000855BB000859BB00085DBB0008B0
:2040800061BB000865BB000869BB00086DBB000893BA000875BB000879BB00087DBB00086F
:2040A00081BB000885BB000889BB00088DBB000897BA00089BBA000899BB00089DBB000866
:2040C000A1BB0008A5BB0008A9BB0008ADBB0008B1BB0008B5BB0008B9BB0008BDBB000850
:2040E000C1BB0008C5BB0008C9BB0008CDBB0008D1BB0008D5BB0008D9BB0008DDBB000830
:20410000E1BB0008E5BB0008E9BB0008EDBB0008F1BB0008F5BB0008F9BB0008FDBB00080F
:2041200001BC000805BC000809BC00080DBC0008DFF8240B40697047DFF81C1B486170477F
:20414000DFF8141B08707047DFF80C0B0078704738B901EBC100052190FBF1F000F5A070D8
:2041600006E001EB8100A0F5C860092190FBF1F000B2704710B5DFF8E44A00206060A06185
:2041800001F0BFFE08B9082005E0042807DB012001F0B1FE0620BDE8104002F02BB80120C3
:2041A00002F028F8DFF87C0EC069606110BD30B583B004460D46062100A802F025FA2A46D0
:2041C0003FA100A802F034FA05F1090100A8DFF8882A12786AB9642D07DA0A2D03DA002DA6
:2041E00005D5002901D443210CE0432113E043210EE0642D09DA0A2D03DA002D07D5002934
:2042000003D445218170202105E0452103E04521417020218170C17000A9204601F0AFF9DF
:20422000DFF8380A1421016037BD70B582B0DFF8F84D60780FF28C0120B9009110236022E3
:2042400000210BE0012802D16068009002E0022808D10091102360220021002002F04EFA58
:20426000606025E0032823D10025542616E01C200FF2F01100FB051060600E21F01D02F089
:2042800064FA6068009010230E220021F0B202F035FA6060F61F0A2002F0E8FB20788642ED
:2042A000E5DA0E3020706D1C062DDEDB002020706078401CC0B2042808BF0020607073BD93
:2042C000256400000000000000000000000000000000000000000000000000000000000055
:2042E000000000000000000000000000000000000000008898BFBF98880000000080808080
:2043000080808000000000000000000000000000000000000000000000000000000000001D
:204320000000000000206060606060609090909090909090909090909090909090909090DD
:204340009090909090606060606060606070F8888482828383838383838282828283838372
:204360008383838282828282868484848484848484848484848484848484828282828282D4
:204380008282FE00000000000000000000000000000000000000000000000000000000001B
:2043A0000000000000000000000000000000000000000090B0FEFEB0900000000080808001
:2043C00080808000000000000000000000000000000000000000000000000000000000005D
:2043E00000000000002060606060606090909090909090909090909090909090909090901D
:020000040800F2
:204400009090909090606060606060606070F88884828283838383838382828282838383B1
:20442000838383828282828286848484848484848484848484848484848482828282828213
:204440008282FE0000F0F00000F0F0F00000FCF8F0E0C080000F0F00000F0F0F00003F1FFD
:204460000F0703010000000000000000000000000000000000000000000000000000000022
:204480000001FFFF01010101010181C67E380080FFFF818101010101000000000020202036
:2044A000E0E0008040402060C04000808080FFFF81808080000000000000008040402020FD
:2044C00020404080000000003F7F448484848484844727000000008040402020204040C094
:2044E0000000000020C3828684848C8C887830000000008040402020204040C000000000E1
:2045000020C3828684848C8C88783000000000000000008080C0602010180C86E0E0E0ECDA
:20452000FCF2F3F1F0F8ECE4E4E2E30100000000000000000080C0402030180CC0C0C0D83B
:20454000F8E4E6E3E1F1D8C8C8C4C603FCFCFC00000000C0382625010101010101010102AE
:204560007F7F7F0609090909090939484848483010080804FCFC00000000C0382625010198
:2045800001010101010102027F7F0609090909090939484848483010080804040000000026
:2045A000000000008080C06030180C8600E0E0ECF4F6F6FBF5E8E8E4E2E2E100000000002C
:2045C00000000000000080C06030180C00C0C0D8E8ECECF6EBD1D1C8C4C4C201FEFEFE80BF
:2045E0004040605854020202020202843F3F3F00010101010107050506020100FEFE804007
:204600004060585402020202020284843F3F0001010101010705050602010000F8B50C469E
:204620008578303DEDB20A2D38BF2A46C578303DEDB20A2D38BF2B4600783038C0B20A2867
:2046400038BF01460026DFF8D45C18200FF2780700FB016C1CF807C006EB050E8EF860C04A
:2046600000FB026C1CF807C08EF890C000FB036C1CF807C08EF8A8C0761C182EE8DB10271B
:2046800044B902230C220821284600F0ABFD05F1D80000E028460026009010230C22002147
:2046A0000C2000F095F8761C082EF5DB7F1EE7D14CB94FF47A7002F0D9F902F08DF8BDE852
:2046C000F14001F08ABDF1BD00E010080810E00000000000000F102020100F000000000055
:2046E000001010F800000000000000000020203F2020000000000000007008080888700063
:20470000000000000030282422213000000000000030088888483000000000000018202092
:2047200020110E00000000000000C02010F800000000000000070424243F2400000000009C
:2047400000F8088888080800000000000019212020110E000000000000E010888818000088
:2047600000000000000F112020110E000000000000380808C8380800000000000000003F2B
:204780000000000000000000007088080888700000000000001C222121221C00000000005B
:2047A00000E010080810E000000000000000312222110F0000000000000000000000000074
:2047C000000000000030300000000000000000007043C0B201F092BF10B582B00FF210000A
:2047E000002400F0F5F9641C062CFAD313BD0000000000C0F038080404040408081C00003C
:020000040800F2
:204800000000000F1F3060404040402030080000000000C0F0180C0404040C18F0C00000CE
:20482000000000071F306040404060301F07000000000004FC1C38E0C0000004FC04000054
:20484000000000407F40000001071E387F00000000000004FCFC84848484E4040C1000006C
:20486000000000407F7F400000000300000000000000000000040404FCFC040404000000A7
:2048800000000000004040407F7F404040000000000000C0F03808040404040C1C00000072
:2048A000000000071F3860404042423E3E0202002DE9F04184B004468846062101A801F062
:2048C000A3FEE4A62246314601A801F0B1FEDFF85C7701AD387828B9642CA8BF432008DA60
:2048E000432004E0642CA8BF452002DA4520A8702020E87001A9012000F06AFEB878411C74
:20490000B9700FF2540100F0F3FD292001F0F6FEB878032804BF0020B870062101A801F0E3
:2049200073FE4246314601A801F082FE387828B9642CA8BF432008DA432004E0642CA8BFE2
:20494000452002DA4520A8702020E87001A9382000F03EFEBDE8FF8100003060C0800000DE
:2049600000000000000000000000180C06030100000000000000000000003060C0803060A9
:20498000C0800000000000000000180C0603190C060301000000000000003060C08030601B
:2049A000C0803060C08000000000180C0603190C0603190C060301000000183060C0800075
:2049C000000000000000000000000C060301000000000000000000000000183060C0983091
:2049E00060C080000000000000000C0603010C0603010000000000000000183060C09830BB
:204A000060C0983060C0800000000C0603010C0603010C060301000010B582B0012808BFE5
:204A20000FF22C0103D0022808BF0FF2E401009100F03EFA012400F0CBF8641C062CFAD38E
:204A40004FF47A7002F012F8BDE8134001F0C5BBE01864E282010101010182E26418E0003F
:204A6000030C1021274E5850584E2721100C0300F00C0201010101020F00000000000000B9
:204A8000030C081010101008060000000000000000601010909090E00000000000000000A1
:204AA000000E11111010081F101800000000000000010101FF000000000000000000000055
:204AC000001010101F10101000000000000000000000000000000000000000000000000057
:204AE0008080808080808080808000000000000001077980008079070100000000000000B4
:204B0000000000071C0700000000000000000000E018040212214181814122120418E00086
:204B2000030C10202844424141422428100C0300F00C0201010101020F0000000000000046
:204B4000030C081010101008060000000000000000601010909090E00000000000000000E0
:204B6000000E11111010081F101800000000000000010101FF000000000000000000000094
:204B8000001010101F10101000000000000000000000000000000000000000000000000096
:204BA0008080808080808080808000000000000000010719E0B00D03010000000000000033
:204BC0000010181700011618100000000000000000901023102200212001C0B201F08EBD72
:204BE00070B582B00FF2780501F088F9022808D00ED304280AD006D3052808BF0FF20C1497
:020000040800F2
:204C000006E02C4604E00FF2901401E00FF2142405F18C00009000F04BF9DFF8EC5B287895
:204C200080B90226142000FB06402838009010230A2200210A20FFF7CBFD761C092EF1DBB1
:204C4000012004E05021102001F07FFD0020287073BD00002564000028030020D83000205D
:204C600001FF00E11FE000FF010000011E0100011E010000006010109090E0000000000E86
:204C8000111110081F1800001010F04020101030000010101F1010000000000010F0201054
:204CA000101010E00000101F10000000101F100000001013F30000000000000010101F1001
:204CC0001000000010F02010101010E00000101F10000000101F100000E010101010F010E6
:204CE0000000007D8A8A8A8A9170000000000080E0F8FE0707FEF8E080000000101C1F1FEA
:204D00001F1F1F12121F1F1F1F1F1C1001FF0100000000000000101F1010101010180400AF
:204D200000C0201010101020C0000007081010101008070010F00010F01000F01000000302
:204D40001C0300031C03000000202020202020202000000000000000000000000107798011
:204D6000008079070100000000071C070000000000C0201010101020C000000708101010C9
:204D80001008070000001010FE1010100000000000000F1010080000001C222141414182CB
:204DA0000700001E081010101008070000C0A090909090A0C000000708101010100804001C
:204DC00010F02010101010E00000101F10000000101F100000202020202020202000000015
:204DE000000000000000000001FF21212121F9030400101F1010101010180400001010F084
:204E00004020101030000010101F101000000000001010F04020101030000010101F101064
:204E20000000000001FF4140404041FF0100101F10000000101F100000001013F30000009C
:204E40000000000010101F10100000000000E010101010F0100000609D8A8A8A8A917000AD
:204E600001FF2010101010E00000101F10000000101F100000202020202020202000000074
:204E8000000000000000000001077980008079070100000000071C070000000000001010C6
:204EA000FE1010100000000000000F1010080000102310220021084601F020BC38B50FF2FE
:204EC000701451EA000213D100250CE0012D05D1009400F048F801F011FC04466D1C022D54
:204EE0003FDA002DF2D1009400F005FB0846F2E7C8B1002935D101280AD104F120000090AD
:204F000010231022502001F0F9FB04F1400015E0022826D1009410231022002001F0EEFB99
:204F200004F1600019E0E1B101290DD104F1200000F018F801F0E2FB04F18000009010236E
:204F40001A46002108460AE002290AD1009400F0D2FA01F0D3FB04F1A00000F003F801F012
:204F6000CDFB31BD00901023102200215020704770B582B0044650250E01F6B20EE0102152
:204F800005F1100001F0E1FB009400F0B4FAE8B201F0B4FB103D192001F068FDB542EEDA37
:204FA00073BD2DE9F0411F48B0F91280DFF8180B0078012803D1414600F053FB80460FF2DD
:204FC000700400212046FFF7D3FF4FF47A7798FBF7F6F6B20FF62835012105EB4610FFF7F2
:204FE000C7FF07FB1688642798FBF7F6F6B2022105EB4610FFF7BCFF032107FB16800A2296
:020000040800F2
:2050000090FBF2F0C0B205EB4010FFF7B1FF042105F5D070FFF7ACFF052104F12000BDE8EB
:20502000F041A5E7800200206031002028030020808040402020101008080404FE0000001F
:205040000000010102020404080810103F0000000000FE04040808101020204040808000DD
:2050600000003F10100808040402020101000000008080C0C06060303018180C0CFE0000CD
:20508000000101030306060C0C181830307F00000000FE0C0C181830306060C0C0808000EF
:2050A00000007F303018180C0C060603030101008080C0C0E0E0F0F0F8F8FCFCFE000000AF
:2050C00000000101030307070F0F1F1F3F0000000000FEFCFCF8F8F0F0E0E0C0C080800019
:2050E00000003F1F1F0F0F0707030301010000002DE9F0411318DFF82482DFF8D4198D7847
:205100005DB90125CD7000250D7108254D7100250D704D7001258D7028E0CD7825BB0E7952
:205120004F7906EB000EAE449EF833E005EB080484F8D8E002EB050EC644F4182C1994F8F6
:2051400033408EF8D8406D1CEDB2AF42E9D27D1C4D71761E0E71EDB20B2D05D10A20487170
:2051600000200871012025E00D7925BB0125CE784F7911E006EB050EC6442C1894F8334094
:205180008EF8D84006EB020EAE44C644EC1894F833408EF8D8406D1CEDB2BD42EAD3781E59
:2051A0004871721CCA70C0B228B901204871092008710020C870BDE8F08110B50021002229
:2051C0000123934003405400042AB9BFC4F10704A340E41FE3405918C9B2521C082AEFDB7C
:2051E000084610BD2DE9F44F82B082465FEA0308DFF8DC580AD1287828B900260027012018
:2052000028706E700CE0AE686F6910E0B8F1010F0BD1687830B90026002728700120687012
:20522000AE7004E0EE68AF6901E02E69EF6900249DF80800484340000090DFF8E09008E0E3
:2052400014F80A00FFF7B9FF04EB090181F8D800641C00988442F3D300229DF80800DFF806
:20526000741803E09DF8083002EB4302009B9A422FD200240AE021F81EA031F81EE04FEA03
:205280001E2A83F8D8A08CF8D8E0641C8442E9D21318E31803EB090C02EB040E0EEB090369
:2052A00093F8D8A09CF8D8B04BEA0A2A21F81EA0B8F1010F06D1002E14BF2AFA06FA0AFAD6
:2052C00007FAD8E7002F0CBF0AFA06FA2AFA07FAD1E7002408E004EB090A9AF8D800FFF7C5
:2052E0006CFF8AF8D800641C00988442F3D31FB9102E08D1002610277F1EB8F1000F04D1CF
:20530000AE606F6108E0761CF7E7B8F1010F07BFEE60AF612E61EF61BDE8F78F0000002050
:205320002DE9FD4E81B08946DFF8AC07B0F91210DFF894572878012802D100F092F9014697
:205340000A2091FBF0F109B2642291FBF2F6F6B202FB161393FBF0FA5FFA8AFA02FB1611BA
:2053600000FB1A10C0B200906878012803D1E8610020286206E0022805D10020E8611020B7
:205380002862002068700020A8610FF2747405E0FFF713FF8BF83801781CA861AF69DFF844
:2053A0003CB7B7EB490F1FDABB4404EB4610385CFFF703FF8BF8D80004EB4A10385CFFF709
:2053C000FCFE8BF8F800009804EB4010385CFFF7F4FE8BF818013819297801290CBF90F8FA
:2053E000E00190F8A001D3E79DF80400C0F1030009FB00F04300E869296ADFF8D82601E0CB
:020000040800F2
:2054000003EB4903062606FB09F6B3422BDA002609E022F81E4032F81E703C0A8AF8D8400D
:205420008CF8D870761C4E45EADA03EB090AB2440AEB0B0C03EB060E0EEB0B0A9AF8D840FA
:205440009CF8D87047EA042422F81E409DF8087027B9002914BFCC408440DAE700280CBF32
:205460008C40C440D5E700201AE006EB0B0494F8D800FFF7A2FE84F8D80094F8F800FFF7BE
:205480009CFE84F8F80094F81801FFF796FE84F8180194F83801FFF790FE84F83801701CB0
:2054A000A861AE69B6EB490FDFDB0BF1D8000121A96100F01FF8A8690007000E01F01EF9E4
:2054C000A969491CA9610529F3DBE869296A50EA010202D019B9102804D1002005E0481E12
:2054E000286201E0401CE861012004B0BDE8F08E01EB401000901023102200217047F8B5EE
:2055000004460D46DFF8D8651421304601F07CF80FF6240724B900230A220121384606E0E8
:20552000012C07D101230A22012107F12000FFF759FE06E0022C04D10A2201213846FFF7E4
:20554000D7FD009610230A220021562001F0D6F80FF2CC7400F04AFE042803D104F10C00B2
:20556000009005E0002D06BF07F1140000900094102306220021502001F0C0F8F1BD38B564
:205580000C46451EEDB2082D0BD3002509E03638C0B20FF26C51FFF7ABFF2801FFF719F927
:2055A0006D1C207898B114F8010B202808BF0A20EFD02D2808BF0C20EBD0A0F130010A2979
:2055C00038BF3038E4D3A0F141010629DFD331BDF8B504460D4600260FF604070DE0142171
:2055E00001FB0070009010230A220021F6B20A2000FB0640FFF7EDF8761C287888B115F8C9
:20560000010B432808BF0B20E9D0452808BF0C20E5D0A0F130010A293ABF3038C0B20A2061
:20562000DDE7F1BD38B50446DFF8AC04B0F91450B0F91210DFF89004007801280BD100F08A
:2056400010F8002C0CBF2918411B09B20120BDE83440FEF77DBD0CB9681832BD481B32BD04
:2056600029460020FEF774BD70B504460D46DFF86804B0F91200DFF850140978012902D1FC
:205680000146FFF7EEFF4FF47A7190FBF1F2642390FBF3F6B6B24DB9201890FBF3F390FBA7
:2056A000F1F080B292B2904209D10AE0001B90FBF3F390FBF1F080B292B2904201D00320C9
:2056C00070BD9BB2B34201D0022070BD012070BDF8B5DFF8F443DFF80054B5F914000A2813
:2056E00004BF0120A081DFF8FC63F068002800F08980606938B10020606100F0FCFB01F08B
:205700006BF8FFF74EFC00F0F0FB40282DD0B0F5807F58D16089B5F9121088421EDA01203D
:2057200060700121A88AFFF79FFF074600F06EF80028FBD10120FFF775FF68826089B5F90E
:2057400012108142B8BF68820220607000F05EF80028FBD100210120FFF7B0FBB5F9120034
:20576000618988422FD101212AE0B5F91200218988421FDA012060700021A88AFFF774FF6F
:205780000746002200F043F80028FAD1FFF74AFF68822089B5F912108842B8BF688202208D
:2057A0006070002200F033F80028FAD100210220FFF784FBB5F912002189884203D1022106
:2057C0000020FFF77BFB40F2051700F08EFB80B1A08940B1F168B94205D3322141430A31ED
:2057E000A982401CA0814FF49670F060002000F07FFBA08930B1F068B84203D20A20A88259
:020000040800F2
:205800000120A081F1BD00009031002001221021384685E52DE9F0474FF00A09B14EAA4CE7
:20582000AD4F00F0E3FC401E072869D8DFE810F00800C5004400F700910094004901E700AA
:205840006069012801D100F057F9207940B900F0DAFF00213846FEF7E1FE0120207107E0DD
:20586000B06928B9706918B1FEF7DFFC3220B061706978B9608A401C608280B2322805D1C5
:20588000208A411E2182C0B200F0ECFE208A08B900F0FCFE01F017FB012803D000F025FBAC
:2058A00000282DD0F86970613320208200F0DAFEBDE8F04700F0E4BE606928B901206061DA
:2058C00000F019FB00F088FF00F098FC8046E078B8F1010F06D008B100F07EFF0020E08175
:2058E000E07023E0E1894B2908BF002804D100F073FF0120E07000E0C0B1B06908B1306825
:20590000DFE000F07FFC0546B7F912A02078012806D1FFF7A5FE05465146FFF7A2FE82463F
:2059200051462846FEF7C4FF3220B0613068002804BFE0780028E3D100F064FC0546B7F945
:205940001200A842B4BF291A411B122900DA0546A6E0BDE8F047BBE66069012801D100F022
:20596000CBF800F0C2FA48F24001401A07D0C03802D0403806D007E0012060710BE002200E
:2059800060710DE0607101E0607910B9FEF724FF0AE0012802D100F036FF05E0022803D1EF
:2059A00001213846FEF73AFE6079032804D0002000F09EFA0320607183E0606910B9012090
:2059C00000F09BF8484F387828B1FFF725F80020387000F001FFB069002872D100F088FB62
:2059E00005462078012802D1FFF73AFE054600F07DF836A10620FFF7C2FD14200DE060694E
:205A000010B9012000F079F86069012804BFB069002856D1FFF7E4F83220B06151E000F0C8
:205A2000F1FB0546B7F91000A842B4BF291A411B1329B8BF054600F0E1FB8046E078B8F1E2
:205A4000010F06D008B100F0C7FE0020E081E07020E0E189322908BF002804D100F0BCFEEE
:205A60000120E07000E0A8B1B06900287FF447AFB7F910A02078012806D1FFF7F1FD0546AB
:205A80005146FFF7EEFD824651462846FEF710FF3220B0613068002804BFE078002810D176
:205AA0002078012802D1FFF7DBFD054600F01EF801F006FA01464046FFF721FDE089401C9C
:205AC000E081BDE8F0870000280300204600000070030020A02E0020800200200000002075
:205AE000D8000020D83000202804002095FBF9F109B20120FEF75BBB0020606100F06CBEDE
:205B0000000000F8FE0301010103FEFCF00000000000003F7FE0808080C07F3F07000000F9
:205B200000000008040406FFFF0000000000000000000000808080FFFF8080800000000053
:205B4000000000060701010181C37F3E00000000000000E0F0D8CCC6C3C0C0E000000000D7
:205B60000000000607818181C1633F1E00000000000000E0C080808181C37F3E00000000F2
:205B800000000000C060380CFFFF0000000000000000060705040484FFFFC48406000000B9
:205BA000000000FFFF8383838383830300000000000000E0C080808080C17F3F08000000AB
:205BC000000000E0F89C8EC2C3C18181000000000000003F7FC080808080C17F3F0000007E
:205BE0000000000F0303030383E33B0F030000000000000080E0781E0701000000000000D9
:020000040800F2
:205C00000000187E7EC381818181677E3C00000000001C7EFFC180808081E37F3C0000008F
:205C2000000078FEC603010101039EFCF000000000000001018383C361713F0F01000000A9
:205C4000000000000000000000000000000000000000000000000000000000000000000044
:205C60000000000000000000F00000000000000000000101010101011F0101010101010009
:205C80000000000000000000000000000000000000010101010101010101010101010100F6
:205CA0000E11110EE0F80C060301010101021E00000000000F3F70C0808080808040200037
:205CC000000000000000C0C0C0C00000000000000000000000003030303000000000000004
:205CE00008142214080202FE06020202C202061E00000000008080FF81810101030000004E
:205D0000C03008040402FAAAFA0204040830C0000718204058A4DBDEDBA458402018070057
:205D200000F0FEFFF000007F7F7F7F00FF0FE1E00FFFFF80BFBF80FF10188CC66363C68C9F
:205D40001810426331180C0C1831634200F01E1FF00000FF8080FF0042C68C183030188C5C
:205D6000C64208183163C6C6633118088C8CC6C68C8CC6C68C8C3131181831311818313141
:205D8000008C8C8C8C8C8C8C8C8C8C8C8C8C8C0000313131313131313131313131313100AD
:205DA00080C0603098CC66333366CC983060C08088CC6633190C060303060C193366CC8813
:205DC000113366CC983060C0C0603098CC6633110103060C193366CCCC6633190C060301DF
:205DE00000E0180404040418E000000F3040404040300F0000000808FC0000000000000019
:205E000040407F4040000000007804040404048870000060504844424140700000380404D0
:205E20008484C830000000384040404040211E00000080601008FE0000000007040444441E
:205E40007F4444000000FC0484848404040000384141404040211E0000C0308884848404E6
:205E60001800000F3140404040211E00001C04048444340C04000000007E010000000000DC
:205E800000708804040404887000001C2241414141221C0000F0080404040418E000003052
:205EA000414242422219070000000000000000000000000000000000000000001C1CC03071
:205EC000080404040830000007182040404020101C120C0202FE8282E20200000000407F64
:205EE00040000300AA4800787047AA4840687047A84948607047A74908707047A4484078DA
:205F0000704770B5044600250A26A34801F02CF94519761EF9D10A20B5FBF0F19C4A40F672
:205F20006373994203D304205070002070BD48439021B0FBF1F100200FF2A82333F8105069
:205F4000A942D56808D2401C042805D20228F5D1002CF3D0A942F6D3401C70BD00208F49CC
:205F60000A68D243920548BF4FF480700968C943490648BF40F0400090B186490A78012AC9
:205F800004BFCA68824207D18A68521C8A60162A06D340F4004002E000228A60C8604860DB
:205FA000704770B57E494A68D3089CB2C5000E781EB94D600120087009E0844234BF041B3A
:205FC000241AA4B23D2C3CBF8018C51A4D60E80870BD38B5002000F03CFD72481021016006
:205FE000192000F047FD704D0A2021E0002000F02BFD69684118AA68824238BF0246AA60CB
:020000040800F2
:20600000EA68904288BF1046E860288801280CD1A868081AE968401AC008FFF7C2FF04461B
:20602000002141F28830E860A96069602888401E288028880028D9D1204632BD5B490A7887
:2060400022B9C000486001220A7007E04A688018931002EB5372A0EBE2004860811000EB49
:206060005170C010704738B500254F4C0A2026E0012000F0E9FC216941186269824238BF9C
:2060800002466261A269904288BF1046A0612088012811D16069081AA169401AC008FFF7BA
:2060A000CDFF40F6E4414843000BA0F5FA75002141F28830A061616121612088401E208028
:2060C00020880028D4D1284632BD10B5FFF781FF0446FFF7C8FF2E49B4F5C87F05D2B0F5C9
:2060E000967F02DA8C60012000E00220087010BD70B50446FFF76DFF0546FFF7B4FF244929
:206100004A8840F6FF739D4202D18B885B1C07E00023A5F6D966B6F5937F34BF521C0022A5
:206120004A808B808A884B883C2A02D353B9032207E01AB90A2B28BF022202D20A2B01D263
:2061400001224A70A4F57A7296235A4340F6B83392FBF3F250328968B4F57A7F08BF0A3AD4
:2061600000D01CB18B18AB42B8BFAD1AB0F5C87FC8BF4FF4C87040F22632691A4FF47A7389
:20618000504303FB010090FBF2F000B270BD0000280400201C3100200028014008080140AE
:2061A00050310020140C0140900300205831002010B5044645F2555000F0E4FF032000F0B0
:2061C000E4FF0A2060434003000C00F0E1FF00F0E2FF00F0E5FF012010BD80B500F0DBFF5E
:2061E000012002BD2C0196005A002800DFF8B00300787047DFF8A81308707047DFF8A00386
:20620000808B7047DFF89803B0F91E00704720220FF2D431DFF88C0300F0CEBFDFF8800347
:2062200000218180C180018141818161C1600F2101820221418201218182704730B5002238
:20624000DFF85C13C880B1F904300446181B08818D6900B2B0F5FA7FBCBF01224519A34225
:2062600005DAE31A1BB2152BA4BF002500228D611F28B4BF002301230C8A4D8A6A438D698C
:206280006A4300FB04228C8AB1F90A50451B6C4303FB04224881012AB8BF002205DB41F243
:2062A00071708242A8BF41F27072CA6090B230BDBB4A9180884204DA091A122904DB002148
:2062C00005E0411A132901DA022100E001219183B4E770B5B44CB24D287801280ED002289E
:2062E00000F0FC80032849D0042800F09880052800F0E380082800F0208170BDFFF7F5FD64
:20630000402811D0B0F5807F18D16878012817D000F05DF9042811DA0320287000202884D3
:206320002060A061606109E06878012808D0022028700020A0610120FFF7DDFD687820B1D4
:20634000E06910B96870FFF7D3FD00F040F940B9FDF7EEFE012804BF0020FDF7EDFE082078
:206360002870A878042818BF012806D0286C60610020FFF7BDFD0120A87070BDFFF7B5FD30
:2063800048F24001401A04D0C03802D040380AD00FE000F016F905202870002060604FF46A
:2063A000FA70E06005E000F054FB00F00DF900F011F900F00CF9042805DB00F002F900F043
:2063C00003F900F007F9B5F93660606848B93046FFF78EFE00F0F0F800B200F03AFB1E20DF
:2063E000606000F03AFB00B9606000F06CFD98B9288C18B901202884E86BA060A0680028C0
:020000040800F2
:206400004DD1A883A06100F024FB0020FFF770FD286C6061042041E0002028843FE0B5F96D
:206420003460B5F93610B142B8BF0E46606848B93046FFF75DFE00F0BFF800B200F009FB39
:206440001E20606000F0C3F804280DDB00F0B9F800F0BAF801202870286C60610420A870F2
:20646000012068703220E061606958B900F0F1FA00F0AAF801206870C820E0610420A870EB
:206480000120287000F01FFD012802D0FFF72DFD28B10020A0616061288403202870FFF704
:2064A0002DFD02287BD3FDF743FE012804BF0020FDF742FE0820287070BDE06800286ED129
:2064C0003A4E0120307001F044F801F095F800203070032028700020206070BDE06920B166
:2064E0000020BDE87040FFF703BDFFF7FEFC48F24001401A12D0C03810D040380BD1FFF7A8
:20650000E4FDFFF7EFFC012803D101F022F801F073F8C820E061E878002840D00020E8701C
:2065200000F097FA012028700220A8700120687000F04AF83220E06170BDFFF7DFFC801E8D
:20654000012803D9801E01280FD921E0B5F93600FFF7CEFDE883FFF7D1FC012818D103207E
:2065600028700020FDF7E8FD12E000F030F801280EDB00F02CF804280ADA00F022F800F050
:2065800023F8012068700220A061A87001202870074820B100F015F806481021016070BDC9
:2065A0005C02002080020020D8300020280400205B6A0008140C0140E8833146B5F91E006B
:2065C00076E6002000F045BA0020FFF794BC0120FFF797BC012028700320A8700120687093
:2065E0003220E06170470000322E3132000000000000000000000000D007B80B6400000090
:2066000050460000A08C0000002201F0BDBD50F8041B61B150F8042BD30744BFA9F10103C0
:206620009A18002342F8043B091FFAD1EFE770470CB41CB5044604A80190009401AB0A46E4
:2066400000A907487844183001F0B8FD009900220A7000285CBF0098001B16BC5DF80CFB3F
:20666000CF0B000080B500A90FF2F42213680B608DF803003C22042100A802F0F3FC01BD13
:2066800000B583B000A80FF2DC2104E000B583B000A80FF2D8210CC90CC03C22062100A830
:2066A00002F0E0FC07BD10B5A0B00C4640218DF80010411CC9B2012000AA03E014F8013B1D
:2066C0008354401C8842F9DB3C2200A802F0CAFC204620B010BD30B583B000AA0FF29423AE
:2066E00030CB30C220308DF8050000A84278891841703C22082102F0B5FC37BD2DE9F041BA
:20670000044690465818C0B2CE080722114218BF761C811000EB5171CA10B0EBC2011ABF6D
:20672000501CC5B2D5B2069F09E031462046FFF7D2FF39464046FFF7B6FF0746761CF6B286
:20674000AE42F2DB3846BDE8F08130B5A1B004460D4601A8FFF758FF00F051F82A46002155
:20676000E0B2FFF7CBFF00F04AF82A460821E0B2FFF7C4FF21B030BD80B54FF48070ADF8E6
:20678000000003208DF8020010208DF8030000A90E4802F0A3FC01BD10B50D4C4FF48071F7
:2067A000204602F002FD022000F060F94FF48071204602F0F8FC022000F058F93C222E2187
:2067C0000448BDE8104002F04DBC0000000C014000080140A002002000B5A1B0802101A8D5
:2067E000FFF712FF00F00BF8802200F0B5F800F006F88022194600F0B0F821B000BD01A8A2
:020000040800F2
:206800000090082370472DE9F041A2B00125002201A90FF2681000F0BCFE040000F07F8065
:206820002078422804BF60784D2840F0878094F83600FF2804BF94F83700FF2804D194F818
:206840003800FF2808BF002500F081F801260F27002000210C2202FB0712121992F83E208F
:2068600080234FF0080C03EA020E1DB1BEF1000F0CD102E0BEF1000F08D00DF1080E864466
:206880009EF8018046EA08088EF8018000F059F8E9D1491C0C29DDD37606360E7F1E082FC1
:2068A000D6DA02A800900823602200F055F8FFF794FC00F04CF801260027002000216FF05C
:2068C0000B0202FB0712121992F8922080234FF0080C03EA020E1DB1BEF1000F0CD102E0F0
:2068E000BEF1000F08D00DF1080E86449EF8018046EA08088EF8018000F023F8E9D1491C9C
:206900000C29DCD37606360E7F1C082FD5DB02A8009008236022082100F01FF808E00FF251
:20692000680000901023602200210020FFF7E6FE4FF47A7000F09AF8FFF74FFC22B0BDE828
:20694000F081401CC0B25B08BCF1010C70477F210DF1090002F056BC00210020CEE6000084
:2069600080818000808D801480AF0000808D801080AE000080B080218020807F4C4F474F5A
:20698000494E2020424D500000000000000000000000000000000000000000000000000041
:2069A00080C0E0F0F8FCFEFEFCF8F0E0C080C0E0F0F8FCFEFEFEFC783080C0C000189CCE2F
:2069C000E6F0F8FCFEFEFCF8F0E0C0E0F0F87C000000000000000000000000000000000029
:2069E000000000000000000000000000000000000000000000000000000000000000001F78
:206A00000F07030103070F1F3F7F7F3F1F0F07030103070703191C0E6773391C0E070301D0
:206A200003070F1F3F7F7F3F1F0F0703010000000000000000000000000000000000000069
:206A40000000000000000000DFF8281431F810007047DFF82414C8607047DFF81C04C06826
:206A600070472021DFF8140402F0CCBBDFF80814142202E0DFF800140A2250438860886829
:206A80000028FCD17047DFF8F8134FF400620A614FF480520A61002808680AD120F44040D1
:206AA00040F440500860086820F4402040F4403009E020F4804040F430400860086820F4D5
:206AC000802040F430200860704780B502F09EFB102002F05FFC012002F056FCDFF8A40353
:206AE0004168DFF8A42311434160016841F080710160012002F0A3FB012002F0A3FB3920B3
:206B000002F011FC0028FAD0022002F09EFB02F0A3FB0828FBD10121172002F0E0FB012103
:206B200040F20C6002F0E4FB0121032002F0E9FB0120BDE8024002F094BB80B501464FF0C7
:206B4000006002F0DAFC4FF4A06002F0A5FC14208DF8000002208DF8010000208DF802002F
:206B600001208DF8030000A802F09BFC01BD38B5C64C4FF6FF70E060C5492160C54961602C
:206B8000C54DE860C54828604FF0883068608020ADF80000002000F01FF84FF4807000F0B8
:206BA00021F80121BE4802F002FB102000F01AF80120ADF80000002000F01AF80220ADF8C4
:206BC0000000002000F014F84FF41070ADF80000482000F001F831BD8DF8030000A920465B
:206BE00002F07CBAADF8000003208DF8020010208DF8030000A9284602F070BA2DE9F041EC
:020000040800F2
:206C000090B04FF420442546A64E304602F08AFCA5480590974806900020079002200890D8
:206C20000020099080200A904FF480700B904FF480600C9020200D904FF400500E900020A6
:206C40000F9005A9304602F0BAFC0121304602F0D1FC964E304600F0DBF900F05FF84FF4CA
:206C6000602702970020039002208DF8100000A9304600F0F6F9DFF83882404600F0C8F9C4
:206C800000F04CF802970020039001208DF8100000A9404600F0E5F90723022207213046D5
:206CA00000F023FA072301220821304600F01DFA052301220921404600F017FA0121304640
:206CC00000F0F6F90121304600F0E9F90121404600F0E5F9304600F0F4F9304600F0F6F94D
:206CE00020B12846451E0028F7D114E0404600F0E8F92546404600F0E9F920B12846451E52
:206D00000028F7D107E00121304600F0E5F90121404600F0E1F910B0BDE8F081002000903E
:206D200001208DF804008DF80500704700B585B04FF4E06002F0B0FB2F20ADF8040042F232
:206D40000F70ADF808000020ADF80A00ADF8060001A94FF0804002F073FC00F061F802F048
:206D6000C5FC012200F05CF802F0B8FC00F058F802F0AAFC1C2000F02AF805B000BD1FB5D9
:206D80004FF4E06002F088FB2F20ADF804003120ADF808004FF48070ADF80A000020ADF85E
:206DA0000600444C01A9204602F04AFC0121204602F09CFC01220121204602F08FFC012199
:206DC000204602F081FC1D2000F001F81FBD8DF8000000208DF8010001208DF802008DF884
:206DE000030000A802F05DBB80B500F019F802F087FC0020304901EB8002536813B15368F2
:206E00005B1E5360401C0828F5DB0878401C08700321084204BFBDE80140FFF79FB801BD74
:206E200001214FF08040704780B50121214802F067FC1148416811B14168491E4160816807
:206E400011B18168491E8160C16802781B4B49B1C168491EC160002A19BF1021596010216E
:206E60001960D243C16811B9102159600022027001BD0000783100200C310020D830002007
:206E800004080140001002400A846800000801408888880883B8BB8B000C01400088834457
:206EA00000013000080002404C240140002401400028014000040040D4300020100C014013
:206EC0005148C089704751480088704700B585B08DF800008DF801101D22022100A802F040
:206EE000C1F80DE000B585B08DF8000003461D22012100A802F0CBF843489DF800100173D2
:206F0000012005B000BD80B500212A20FFF7DEFF02210E20FFF7DAFF03212A20FFF7D6FF12
:206F200000212B20FFF7D2FF01212A20BDE80440CCE770B51C460023002500F11006964268
:206F4000A6BFA0F11006B242012301F11006A642A6BFA1F11006B442012300F12006964207
:206F6000A6BF20388242012501F12000A042A6BFA1F120008442012524480580184670BDF7
:206F800021480178407802E01F480179407940EA01200009802903D3C043401C0005000D97
:206FA000704730B583B0184C06212046FFF72CFB0020FFF797FFE8B1207B00071AD50120FD
:206FC000FFF790FFB0B1207B8DF80000207000A8417861709DF8021021719DF80310617136
:206FE0000179217240796072FFF7CAFF0546FFF7CBFF00E0258A00232A460021208AFFF74C
:020000040800F2
:2070000098FFE081258237BDF83000200A31002080B55749884208D101214FF4007002F0FB
:2070200079F900214FF4007016E05249884208D101214FF4806002F06DF900214FF48060F5
:207040000AE04D4988420BD101214FF4004002F061F900214FF40040BDE8044002F05AB987
:2070600001BD4268454B1A400B681A430B7942EA032242608268424B1A40CB681A438B6823
:207080001A434B7942EA43028260C26A22F47002097C491EC9B242EA0151C16270470029E0
:2070A000816812BF41F0010149084900816070470029816814BF41F4807121F480718160BF
:2070C0007047816841F00801816070478068C008FFE700F0010070470029816814BF41F4E6
:2070E000A00121F4A0018160704770B507240A290BD3A1F10A0505EB4505C668AC4026EA3B
:207100000404AB402343C36008E001EB41050669AC4026EA0404AB40234303611F23072A3E
:207120000AD2521E02EB8202446B934024EA030391401943416370BD0D2A0AD2D21F02EB0D
:207140008202046B934024EA030391401943016370BD0D3A02EB8202C46A934024EA0303CA
:2071600091401943C16270BDC06C80B2704700000024014000280140003C0140FFFEF0FF46
:20718000FDF7F1FF09490860704709490860704708490860704705484AF6AA210160704749
:2071A00002484CF6CC4101607047000000300040043000400830004062B38B0708D0521ED3
:2071C00011F8013B00F8013B00F024808B07F6D1830740F0208000BF103A07D330B4B1E88F
:2071E0003810103AA0E83810F9D230BC530724BFB1E80810A0E8081044BF51F8043B40F825
:20720000043BD20724BF31F8022B20F8022B44BF0B7803707047083A07D3B1E80810083A19
:2072200040F8043B40F804CBF7D25307E4E70268531C03601170704770470000F8B5642482
:20724000DFF8742C0A23072911D8DFE801F0041123588090C5CC017845785D4304FB015161
:207260008078401841F2D041401A58431082F1BDDFF8481C09780029F9D1017845785D43C0
:2072800004FB01518078401841F2D041401A58435082F1BDC17846788578A1F1300C5FFA79
:2072A0008CFCBCF10A0F0CD200784FF47A77664307FB006003FB0500081800F53C57B03759
:2072C00018E0A5F13001C9B20A2909D2007803FB06F104FB0010281841F2D041471A09E01C
:2072E000A6F13001C9B20A2904D2007803FB0060A0F504773FB204FB07F09061F1BDC1789D
:207300008578A1F13006F6B20A2E0DD206784FF47A774078604307FB060003FB05000818B1
:2073200000F53C57B0370DE0A5F13001C9B20A2908D201784078584304FB0100281841F263
:20734000D041471A3FB204FB07F0D061F1BD46780778A6F13000C0B20A283ABF03FB0760EF
:20736000A0F50477303F03FB07F09082F1BDC178467807788578A1F13000C0B20A280CD222
:207380004FF47A7004FB06F200FB072003FB0500081800F53C57B03717E0A5F13000C0B2E6
:2073A0000A2808D203FB06F004FB0700281841F2D041471A09E0A6F13000C0B20A283ABF95
:2073C00003FB0760A0F50477303F3FB203FB07F0DFF8EC1A0860F1BD00783038C0B2BDE8F9
:2073E000F240FCF7ADBE467807788578A5F13000C0B20A2808D203FB06F004FB0700281845
:020000040800F2
:2074000041F2D041471A09E0A6F13000C0B20A283ABF03FB0760A0F50477303FDFF89C0A19
:20742000007818B9DFF89C0A3FB20760F1BD000030B507291DD8DFE801F004041E324151D4
:2074400060658378A3F13001C9B20A293FBF4478A4F13001C9B20A2979D20178A1F1310044
:20746000C0B2042873D2342903D1302C08BF302B6DD1012030BDC1783039C9B20A2921BFFE
:2074800081783039C9B20A29F3D341783039C9B20A295CD200783638C0B2042828E0C17853
:2074A0003039C9B20A29E4D381783039C9B20A294DD200783338C0B2072819E00178407821
:2074C0003038C0B2062804D2A1F13000C0B203280EE03529CDD2312939D1CAE7017840783E
:2074E0003038C0B2032805D2A1F13000C0B20A28BFD32CE03929BCD229E001783129B8D058
:207500003029E9E74478017883780A20A3F13005EDB20A2D08D26425604305FB0100181812
:2075200041F2D041401A0AE0A4F13003DBB20A2B3ABF00FB0140A0F50470A1F13000012A0E
:2075400097D180B2DFF87C190968884291D0002030BD10B54FF41852DFF86C19DFF86C0962
:20756000FFF73AFEDFF86809002100220B460C461EC010BD10B5002208E0135CA3F16104CD
:20758000E4B21A2C3CBF203B1354521C8A42F4DB10BD2DE9FF4180460E46DFF8304904F2C6
:2075A000004710250B22394601A8FFF705FE0B2101A8FFF7DFFF0B22414601A802F0B8F859
:2075C00098B907F11C00017831704178717007F11A0000A902780A7042784A70BDF80000BA
:2075E00004EB402000F5007003E020376D1ED9D1002004B0BDE8F0812DE9F04FADF5097D01
:207600000024ADF8004000260FF6E80700AA0DF102013846FFF7BDFF0190DFF8B09809F2C1
:2076200000400290DFF8A8A80198002800F001814FF48C7143A8FEF7E7FFDFF898784FF4EE
:20764000007201993846FFF7B7FDA0460025232043A900FB081B05E0232D3CBF05F80B0066
:207660006D1C761C384602F095F8864206D2F05D0D2802BFF11949780A29EDD105F80B400B
:20768000B61C08F10108B8F1080FDFD30027DFF828880AEB87056E69304602F07BF823217F
:2076A00043AA01FB072B02463146584602F040F800286CD1686902F06DF8064604E0202823
:2076C00018BF3D285DD1761C00F0C3FA864258D216F80B00A0F13001C9B20A29EFD230286D
:2076E00001D1062F4DD15E440022F9B23046FFF79FFE002845D0F9B23046FFF79FFD2FB915
:20770000B8F9100000F097FA43A837E0012F05D1B8F9120000F089FA4BA81DE0022F06D1F1
:20772000D8F8180000F075FA0DF5A97026E0032F05D1D8F81C0000F066FA5DA81DE0042F68
:2077400005D1B8F9140000F06AFA66A816E0052F04D100F076FA6EA8C01C0FE0062F07D1DF
:20776000FCF7F2FC02460FF2F0710DF5EF7005E0072F16D100F042FA80A8401CFEF758FF1F
:207780000FE000F066FA0146584601F03BFD6C6B204601F0FFFF024621465846FFF70CFD24
:2077A00001247F1C082FFFF474AF002C02BFDFF80C07007800283BD0FE2103A8FEF724FF58
:2077C0000027232043A900FB071103A801F0FDFF0AEB8700416D03A801F0F7FF7F1C082F1A
:2077E000EFD303A801F0D6FF0246BDF8000009EB4010FF2A80F81C2400F21C4094BF002172
:020000040800F2
:20780000110A417001980299401A00F50070411200EB91508012012100F80A1003A801F028
:20782000B9FF024603A90198FFF7C6FC00F058FA5DE00FF2407500AA0DF102012846FFF707
:20784000A8FE09F21644DFF89086D0B1FE22014603A8FFF7B1FC00F05CF809F584600ECD09
:207860000EC0FE2203A909F50060FFF7B5FC6675C4F82080032089F83A04FE2089F83C0471
:2078800001E000F046F802980ECF0EC00FF6F007062239464846FFF79FFC0622394609F52D
:2078A0000070FFF799FC00270AEB8705D5F834B000F0CFF900F032F8686B01F06BFF8619D5
:2078C000D5F854B000F0C5F900F028F8686D01F061FF86197F1C082FE6D3002089F80B0419
:2078E000C9F8168402202071A67100F022FA42F60C0000EB09010022CA760A774A7640F843
:207900000920002088600861C8600DF5097DBDE8F08F4FF418514846FEF776BE02465946AF
:2079200006EB090000F5C060FFF746BC2DE9F04FADF50B7D06460F46DFF89455DFF88C9568
:20794000B7F5805F0BD14FF40072494601F0F0FE002815D04FF40072314648460CE0B7F53E
:20796000205F0ED109F5007400F076F9002807D04FF4007231462046FFF71EFC012028707E
:2079800036E1B7F5804F22D109F2004400F064F90028F5D04FF4007231462046FFF70CFC59
:2079A0000120687010240FF24C570C22314600A8FFF702FC0B22394600A801F0B9FE10B9F0
:2079C000B07E288214E12036641EEED110E1A7F50044B4F5005FF9D807EB0900A0F5F448CD
:2079E0004FF400724146304601F0A2FE08B100F038F9A7F5FC4005EB902A600A801C298A2F
:207A0000884240F0EF8000244FF48C7145A8FEF7FBFDDFF8C08400F024F900260027232007
:207A200045A900FB061B05E0232F3CBF07F80B007F1C641C404601F0ADFE844208D214F817
:207A400008000D2802BF04EB080149780A29EBD1002007F80B00A41C761C082EDED30026F7
:207A6000DFF8547405EB8604D4F814B000F0F1F80246232045A900FB06185946404601F0DC
:207A800057FE002840F09780606901F083FE044604E0202818BF3D2810D1641C404601F05D
:207AA00079FE844280F0A68014F80800A0F13001C9B20A29EDD2302802D1062E40F09A8007
:207AC00044440122F1B22046FFF7B2FC00287BD0F1B22046FFF7B2FB404601F05BFE014618
:207AE000404601F08FFB2EB9B7F9100000F0A3F845A835E0012E05D1B7F9120000F095F80D
:207B00004DA81BE0022E05D1B86900F082F80DF5AD7025E0032E04D1F86900F074F85FA8F6
:207B20001DE0042E05D1B7F9140000F078F868A816E0052E04D100F084F870A8C01C0FE0BF
:207B4000062E07D1FCF700FB02460FF20C410DF5F37005E0072E05D100F050F882A8401C82
:207B6000FEF766FD761C082EFFF47CAFFE2105A8FEF74AFD0026232045A900FB061105A8A9
:207B800001F023FE05EB8600416D05A801F01DFE761C082EEFD305A801F0FCFD0446288AD9
:207BA00009EB4010FF2C80F8DC4300F5777094BF0021210A09E0646B204601F0EBFD024605
:207BC00021464046FFF7F8FA14E041704FF4007205A909F5C060FFF7FFFA012068708AF840
:207BE000010005E0012068708AF8010000F078F800F076F80DF50B7DBDE8F08FB148026854
:020000040800F2
:207C00000FF2643170476421B0FBF1F20FF21C3170476421B0FBF1F20FF2003170470A21D8
:207C200090FBF1F20FF2143170470A2190FBF1F20FF2DC2170470A2190FBF1F20FF2C02110
:207C400070479F4800680A21B0FBF1F20FF2F8217047584601F09EBD4FF40072214601F09D
:207C600067BD4FF4007231464046FFF7A5BA38B504460D46FFF7E0FA25B94FF400720FF2EB
:207C8000003121E09149B5F5805F08BF4FF400721AD0B5F5205F04D14FF4007201F50071CF
:207CA00012E0B5F5804F04D14FF4007201F580610AE0A5F50040B0F5005F0AD84FF4007299
:207CC00005F1006101F58C412046BDE83840FFF773BA4FF400712046BDE8344001F092BA74
:207CE000F8B501F061FB00207949425CD2B1002242548402744D281901F087FD73482618D9
:207D0000002736F8021B3819281801F06DFD042803D001F053FB0420F2BDBF1CB7F5806F7E
:207D2000EFD302E0401C1028DFD301F047FB0020F2BD70B5654C01F037FB0025624E06EB98
:207D4000852001F062FD6D1C092DF8DB002534F8021B701901F048FD042801D0042070BD21
:207D6000AD1CB5F5185FF2DB01F028FB002070BD2DE9F04142F61804544D6619574F327ADE
:207D80002AB9400238604802786001203072307A012831D1605978B905F5185839684046F1
:207DA000FFF765FF40229821404601F043FD4FF4E070605140200CE040229821B868401973
:207DC00000F5185001F036FD605940386051B8684030B8604021012001F0D7FD30210120DF
:207DE00001F05DFD3868403038607868403878603B48816840398160786838B96051B86000
:207E0000386038480321017000203072BDE8F0812DE9F04142F61C042C4D62594032661919
:207E2000314F33792BB9400238604802786001203071307901282FD100202C490AE05B19AF
:207E400003F5185310F801C083F800C0401C63595B1C635163599342F1D3DFF89480B8F888
:207E600000003968411839607A68101A7860C00507D100206051A1F5007105F51850FFF7BE
:207E800055FD17488168B8F80020891A81604FF44051022001F014FD786800281EBF1148BE
:207EA0000078042806D100206051012101F0D4FE00203071BDE8F0818002002028040020CC
:207EC000340400203004002000C0000864040020E8010020A02C0020188DDD403C31002062
:207EE0002C310020A03000204831002040300020A2300020434F4E46494720205458540004
:207F0000545F5374616E6462793D256400000000545F576F726B3D25640000005761697462
:207F20005F54696D653D25640000000049646C655F54696D653D256400000000545F5374E1
:207F400065703D25640000005475726E5F4F66665F763D256400000054656D7053686F7791
:207F6000466C61673D2564005A65726F505F41643D2564004C4F474F494E2020424D500020
:207F8000EB3C904D53444F53352E3000020108000200025000F80C000100010000000000AC
:207FA00000000000000029A298E46C4E4F204E414D4520202020464154313220202033C916
:207FC0008ED1BCF07B8ED9B800208EC0FCBD007C384E247D248BC199E83C01721C83EB3ACE
:207FE00066A11C7C26663B07268A57FC750680CA0288560280C31073EB33C98A461098F74E
:020000040800F2
:20800000661603461C13561E03460E13D18B7611608946FC8956FEB82000F7E68B5E0B03F7
:20802000C348F7F30146FC114EFE61BF0000E8E600723926382D741760B10BBEA17DF3A66B
:208040006174324E740983C7203BFB72E6EBDCA0FB7DB47D8BF0AC9840740C487413B40E36
:20806000BB0700CD10EBEFA0FD7DEBE6A0FC7DEBE1CD16CD19268B551A52B001BB0000E828
:208080003B0072E85B8A5624BE0B7C8BFCC746F03D7DC746F4297D8CD9894EF2894EF6C601
:2080A00006967DCBEA030000200FB6C8668B46F86603461C668BD066C1EA10EB5E0FB6C890
:2080C0004A4A8A460D32E4F7E20346FC1356FEEB4A525006536A016A10918B4618969233AA
:2080E000D2F7F691F7F64287CAF7761A8AF28AE8C0CC020ACCB80102807E020E7504B4429F
:208100008BF48A5624CD136161720B40750142035E0B497506F8C341BB000060666A00EBC3
:20812000B04E544C44522020202020200D0A52656D6F7665206469736B73206F72206F7484
:20814000686572206D656469612EFF0D0A4469736B206572726F72FF0D0A50726573732064
:20816000616E79206B657920746F20726573746172740D0A00000000000000ACCBD855AAC1
:20818000F8FFFFFFFFFF000000B500BF130096469446103928BFA0E80C50FAD85FEA417CC3
:2081A00028BF0CC048BF40F8042BC90728BF20F8022B48BF00F8012B00BD00002DE9F04F65
:2081C000A1B0804617461D46029102AE0020706211AC6FF000490AE017F8011B0298C04778
:2081E0000290002800F06A82706A401C7062387808B9706A64E22528EED10020F060306143
:208200007061B061F061306201E040F0010017F8011F2029F9D023290DD02B2904D02D299F
:2082200006D030290AD00CE040F0020080B2EEE740F00400FAE740F00800F7E740F01000A5
:20824000F4E72A290DD129680A1D2A600968F162002904D54942F16240F0040080B27F1C2B
:2082600012E00021F16209E0F16A494505D001EB810302EB43013039F1627F1C3A78A2F1B4
:208280003001C9B20A29EFD339782E2903D04FF0FF31B1621DE017F8011F2A2906D12968F9
:2082A0000A1D2A600968B1627F1C12E00021B16209E0B16A494505D001EB810302EB4301C0
:2082C0003039B1627F1C3A78A2F13001C9B20A29EFD3308639780FF6983001F0FFFC08B1C8
:2082E00017F8010B8DF83A009DF83A00682804D1387868280AD1622005E06C2804BF3878E7
:208300006C2803D171208DF83A007F1C11A8B0603978B1F1250023D01C3871D0001F0228F8
:208320006ED9133800F09680093869D0801E00F02781401E00F0D180401E022860D9001F76
:2083400000F0CB80401F30D0401E00F08380401E20D0C01E09D0801E7CD0C01E7AD017E123
:20836000F068411CF16025211BE12868011D296000687060B26A002A02D501F00BFA07E04C
:20838000002101F0B7FC00281ABF7168401AB06A306107E12868011D296000680021CDE9DB
:2083A000000111A870607821E6E09DF83A00622818D0682806D06A280BD06C2819D07128AA
:2083C00007D016E02868011D2960716A00680180E8E02A68101D2860706AC1171268C2E9EF
:2083E0000001DFE02868011D2960716A00680170D8E02868011D2960716A00680160D1E08E
:020000040800F2
:208400002868C01D20F00700286000F108022A60D0E90023CDE90023002B04D5F068421C5C
:20842000F2602D220DE0308E820704D5F068421CF2602B2205E0C00704D5F068421CF260AC
:2084400020220255F06811AA8018706000A800F0C5F9A7E09DF83A006C2808BF2A6811D08E
:20846000712808BF2A6802D06A282A680AD1D21D22F007022A6094460CF108022A60DCE975
:20848000002303E0131D2B6012680023CDE90023682808BF92B207D0622808BFD2B203D08B
:2084A000742818BF7A2802D10023CDE9002396F8300000075CD5DDE90023002B08BF002ADD
:2084C00056D041F02000782852D1F06830220255401C421CF26001554AE09DF83A0062287C
:2084E0000CD0682810D06A281AD06C2823D0712816D074281FD07A280CD01CE02868021DFA
:208500002A6090F900201AE02868021D2A60B0F9002014E02868021D2A60026800230FE083
:208520002868C01D20F00700286000F108022A60D0E9002304E02868021D2A600268D3175D
:20854000CDE90023002B04DAF068421CF2602D220DE0308E820704D5F068421CF2602B2280
:2085600005E0C00704D5F068421CF26020220255F06811AA8018706000A800F0A4F811E035
:20858000F068411CF16029680A1D2A60096808E0F068421CF2602522025519B1F068421C14
:2085A000F26001557F1CF06AF168401AB169401A3169401AF169401A7169401A316AA0EBF5
:2085C000010A96F83000400711D420208DF84000BAF1010F0BDBD346012310AA00A94046DA
:2085E00000F02FFC002869D1BBF1010BF4D1F36811AA00A9404600F024FC00285ED1302085
:208600008DF84000D6F818B0BBF1010F0ADB012310AA00A9404600F014FC00284ED1BBF15E
:20862000010BF4D13369726800A9404600F009FC002843D130208DF84000D6F81CB0BBF138
:20864000010F09DB012310AA00A9404600F0F9FBA0BBBBF1010BF5D17369306971684218B4
:2086600000A9404600F0EDFB40BB30208DF84000D6F820B0BBF1010F09DB012310AA00A91E
:20868000404600F0DEFBC8B9BBF1010BF5D196F8300040077FF5ABAD20208DF84000BAF10B
:2086A000010FFFF6A4AD012310AA00A9404600F0C8FB18B9BAF1010AF5D198E54FF0FF306C
:2086C00021B0BDE8F08F2DE9FA4782B0064635696F2908BF082705D041F02000782814BF0B
:2086E0000A2710273C24D6E90001804689469DF80820642A18BF692A05D1002903DAD8F103
:20870000000869EB4909B9F1000F08BFB8F1000F0CD1306B50B9082F3BD196F838000007E2
:2087200037D53B24302085F83B0032E0A4F1010A5446FB17404649463A4601F007FBCDE92A
:208740000089B846A8FB0023DDE90089A8EB02023032D2B23A2A03D39DF80830513B9A18BB
:208760000AF8052080465FEA010908BFB8F1000F03D0F06861198842D8D3082F09D196F881
:208780003800000705D5605D302802D0641E30206055C4F13C00B0616119F160316B88421F
:2087A00007DA081A3062308F4FF6EF710840308710E000290ED596F8381001F014011029B0
:2087C00008D1716B7269891A326A891A081A0128A8BF306204B0BDE8F08700002DE9F24FBC
:2087E0008EB0044604AED4E90001CDE902019DF8380040F020008DF8000061280BD0206B37
:020000040800F2
:20880000002848BF062005D404BF9DF80000672801D1012020636168C1F30A5040F2FF7352
:2088200098421ED1080304BF206800280AD10320A0619DF838006138C0B21A2838D30FF2CC
:20884000446109E00320A0619DF838006138C0B21A282AD30FF224610322E068FEF7ACFCBF
:20886000B9E1012817DA204601F0E7FA012812DB002700209DF80010612920D1E1683022F4
:2088800001F8012B4A1CE2609DF83820612A0CBF782258220FE040F2FE31626861F31E52D6
:2088A0006260471A4FF0FF30E4E70FF2CC51D3E70FF2CC51D0E70A706169891C616110B93B
:2088C000002500277EE19DF80000612840F09780206B00284CBF2125451C2DB26E1CD4E9FD
:2088E0000089DDE902010022002301F0C7FA3ABF89F00040CDE90280CDE902893F1F8DF821
:2089000010200DF11108012E35DBDDE902010022002301F0CBFA2ED21C2102A801F0DEFA5D
:20892000DDE9020101F060FB8146F61F012E09DB01F086FB02460B46DDE9020101F098FBDB
:20894000CDE9020108F20700072105E009F00F0200F8012D4FEA2919B9F1010F01DB491EA8
:20896000F4D5491E5CBF002200F8012DF9D500F20708012EC9DA0DF11100A8EB00010DF122
:208980001106A942B8BF0D462DB2002D30D42846884206DA04A941184978082928BF0F21D4
:2089A00000D2002104AA821800E06D1E401E12F801398B42F9D00F2904D104A941184A7804
:2089C000521C4A70002802D504AE6D1C3F1D2DB2681E0DD481190A783032D2B23A2A03D357
:2089E0009DF838303A3B9A1801F80129401EF2D5206B002840F1E680681E2063E2E0DDE930
:208A000002010022002301F039FA3CBF81F00041CDE902013FB247F297507843474990FB9D
:208A2000F1F73FB2C7F107069246DFF814B1012E19DBDDE90289F00707D552465B4640461E
:208A4000494601F0D5FB8046894676105046594652465B4601F0CCFB82468B46002EEAD103
:208A6000CDE9028921E076429046DFF8D89012E0F00707D552465B464046494601F0B8FB30
:208A80008046894676105046594652465B4601F0AFFB82468B46002EEAD1DDE902014246DF
:208AA0004B4601F077FCCDE902019DF8000066280CBF07F10A000620216B4518142DA8BF61
:208AC000132530208DF810000DF11106DFF87890012D3BDBDDE9020101F09CFA06F10801F1
:208AE00004220A26B0FBF6F303EB830EA0EB4E00303001F8010DB3FBF6F000EB8006A3EB3A
:208B00004603303301F8013D521EEAD101F10806083D012DDCDBDDE9020101F07BFA01F0FD
:208B200099FA02460B46DDE9020101F0A1FA00224B4601F05DFBCDE90201CBE7A086010026
:208B4000000024400000F03F84D797410DF11100301A0DF1110602E0401E7F1E761C3178C9
:208B60003029F9D09DF80010662902D13FB2791C03E065290CBF01210021226B8D182DB2B6
:208B8000A842B8BF05462DB2002D1BD42946814204DA885D352828BF392000D230208A19D7
:208BA000521E00E06D1E491E12F801398342F9D0392802D1885D401C8855002902D5761EBB
:208BC0006D1C7F1C3FB200972BB232469DF83810204600F003F80FB0BDE8F08F2DE9F0433A
:208BE00085B00546894617461E46D5F83080012E02DA01260FF2902749F02000BDF930407F
:020000040800F2
:208C0000662808BF641C18D0672840F082806FF003008442C0F28380444580F28080641C7E
:208C200095F83800000702D44645B8BFB04624B2B8EB040848BF4FF00008E868A96924B28F
:208C4000012C25DA4A1C30230B54B8F1010F03DA95F83810090702D52E211154521CAA6151
:208C600018EB040FB8BFC8F1000424B261426962A044B045B8BF464636B2EE61324639465C
:208C8000AB691818FEF798FAA8EB0600A862C1E00818A64218DA32463946FEF78DFAA96946
:208CA0007118A961A01B6862B8F1010F03DA95F83800000705D5E8682E220A54E869401CB5
:208CC000E861C5F82880A5E022463946FEF774FAA8692018361BB8F1010F03DA95F8381012
:208CE000090703D5E9682E224254401CA86136B2B045B8BF464636B23246E119EB68C0188B
:208D0000FEF75AFAA8693018A861A8EB0600686280E0B9F1610F16D14FF0700918E04645A9
:208D200004DA95F83810090758BFB046B8F1010848BF4FF00008B9F1670F14BF4FF04509E3
:208D40004FF0650904E0B9F1410F08BF4FF05009A9694A1CE86817F8013B0B54B8F1010FFE
:208D600005DA95F83810090758BFAA6117D52E211154531CAB61B8F1010F10DB761E36B2D2
:208D8000B045B8BF464636B2324639461818FEF713FAA8693018A861A8EB06006862A869F4
:208DA000E968471807F8019B002C03D42B2007F8010B03E02D2007F8010B644200260DF10A
:208DC000080809E00A22214600A801F006FC019808F8010B009C761C24B2012CF2DA022E9A
:208DE00006DA49F02000652804BF302007F8010B4EB9302007F8010B07E0761E02A8305C7C
:208E0000303007F8010B012EF7DAA869E9684018381AE86195F8380000F0140010280DD1B3
:208E20006869A9690818696A0818E9690818A96A0818696B8842BCBF081A286205B0BDE878
:208E4000F083F8B504460D4616461F46002077B116F8011BA868A047A86030B1E86A401C94
:208E6000E86200207F1EF3D1F2BD4FF0FF30F2BD686A6C747A4C00006E616E004E414E00C9
:208E8000696E6600494E460030000000002800E0401EFDD1704710B586B0FDF76DFCC02065
:208EA000ADF8000003208DF802001C208DF8030000F04CF80020ADF808004BF6FF70ADF849
:208EC0000A003C20ADF80C004FF48060ADF80E004FF48040ADF810005F4801905F4C01A960
:208EE000204601F081FB0121204601F0DDFB06B010BD5B4A012903D10146104600F053B98F
:208F000019B90146104600F050B9704780B50121082000F0EDF9C020ADF8000014208DF89F
:208F2000030003208DF8020000F010F800F012F800F05BF800F05CF800F055F8002100F0BD
:208F400055F800F050F800F005F801BD00A9444800F0C4B800214020CBE780B5FFF7FAFFE9
:208F6000002100F043F800F03EF800F041F800F03AF800F03AF800F036F8FFF7EBFF0220F2
:208F8000BDE8024082E738B50446082508E000F02DF800F028F800F02BF800F024F864008D
:208FA0002846451EC0B230B1FFF7D4FF20064CBF01210021EBE7FFF7CDFF00F016F8FF249B
:208FC00000F011F800F043F848B900F011F800F00AF8FFF7BFFF00F006F8012032BD641E4D
:208FE000EED1002032BD022050E70121802080E7012140207DE770B5044608250026FFF783
:020000040800F2
:20900000F4FF0DE0FFF7A6FFFFF7EDFFFFF7F0FFFFF7E9FF760000F01AF808B146F00106C2
:209020002846451EC0B20028ECD1FFF793FF002C0CBF01210021FFF7D9FFFFF7D4FFFFF7B9
:20904000D7FFFFF7D0FFFFF785FFF0B270BD8021034800F0A1B80000A0860100005400403C
:20906000000C014070B504460D461646FFF74EFF7000C0B201E014F8010BFFF784FF284680
:20908000451EC0B20028F6D1BDE8704065E7F8B504460D4616461F46FFF738FF7600F0B21B
:2090A000FFF771FF3846FFF76EFFFFF72FFF46F00100C0B2FFF767FF03E0FFF79CFF04F8D0
:2090C000010B2846451E28B1EDB2002D0CBF00200120F2E7BDE8F1403FE700002DE9F041E6
:2090E0000022CC7804F00F03E40644BF8C7823430C8801250F26E7B217B3D0F800C005FAD4
:2091000002F7BE460EEA0408F04514D14FEA820E06FA0EF82CEA080C03FA0EFE4EEA0C0CE2
:2091200091F803E0BEF1280F08BF476103D0BEF1480F08BF0761521C082AE0D3C0F800C09B
:20914000B4F5807F26D3D0F804C0002202F1080705FA07F7BE460EEA0408F04515D14FEA65
:20916000820E06FA0EF82CEA080C03FA0EFE4EEA0C0C91F803E0BEF1280F08BF476191F88C
:2091800003E0BEF1480F08BF0761521C082ADDD3C0F804C0BDE8F08100228068084218BFAA
:2091A000012210467047016170474161704770B5134A00284CBF94691468C0F3034583B2AF
:2091C000460D3601B34000F44016B6F5401F06D124F07064156825F07065156008E0C60273
:2091E00043BF032606FA05F5AC439C4344F0706401B11C43002801D5946170BD146070BDA2
:2092000004000140002201F059BA00005048016841F00101016041684E4A114041600168B2
:209220004D4A11400160016821F480210160416821F4FE0141604FF41F018160704747497C
:209240000860704747490860704745490A68920850EA8200086070474148006800F00C00DE
:20926000704741490860704730B53D490A683F4B02F00C02082A0ED10A680C68C2F38342B6
:20928000921C3B4D5543E40302D50C68A40301D52B4600E0534303600B68364A0468C3F3F2
:2092A00003139B5C24FA03F343600B684468C3F302239B5C24FA03F383600B684468C3F32D
:2092C000C2239B5C24FA03F3C3600968C368C1F381318918097CB3FBF1F1016130BD264A04
:2092E0000029116814BF084321EA000010607047224A0029116814BF084321EA00001060D5
:2093000070471F4A0029116814BF084321EA0000106070471B4A0029116814BF084321EA0B
:2093200000001060704700214209094B012A08BF1A6803D0022A0CBF1A6A5A6A012300F0AC
:209340001F0003FA00F0024218BF012108467047001002400000FFF8FFFFF6FE0000424200
:209360000410024060004242D800424200127A0000093D001404002014100240181002407D
:209380001C1002400C100240DFF8D4100A6802F0380206E0DFF8C8100A6822F010020A6013
:2093A0000A68104308607047FFE7DFF8B800DFF8B8100160DFF8B41001607047FFE7DFF8E4
:2093C000B000016841F080010160704738B5054600F015F804280DD1DFF89440206840F008
:2093E00002002060656000F006F8216841F6FD721140216032BD206840F0400020604FF48D
:020000040800F2
:20940000302039E070B504460D4600F011F804280CD1174E306840F001003060258000F0CC
:2094200007F8316841F6FE721140316070BD08804FF4005020E00F490860704704200D49D2
:209440000A68D20701D5012070470A68520701D5022070470968C90648BF03207047000078
:20946000002002400420024023016745AB89EFCD102002400C20024010B5FFE70446FFF799
:20948000DDFF03E02CB1FFF7D9FF641E0128F9D004B9052010BD00001B4908431B490860C4
:2094A000704770B503781A460121C478ECB1174B1B6803F4E063C3F5E0631B0A4478C3F14B
:2094C0000405AC4085780F2626FA03F32B4023431B010F4C1355007842110E4B00F01F006C
:2094E00001FA00F043F8220070BD50110A4A03F01F03994042F8201070BD084A11400843CF
:2095000007490860704700000000FA050CED00E000E400E000E100E080E100E080FFFF1FA1
:2095200008ED00E001684FF6FE72114001600021016041608160C1603349344A90421DD0A8
:20954000334A904221D0334A904225D0324A904229D0324A90422DD0314A904203D1086864
:2095600040F4700029E02F4A904203D1086840F0706022E02C492D4A904203D1086840F07B
:209580000F001AE02A4A904203D1086840F0F00013E0284A904203D1086840F470600CE0AD
:2095A000254A904203D1086840F4704005E0234A904203D1086840F470200860704702688D
:2095C0006FF30E128B681A430B6A1A430B691A434B691A438B691A43CB691A434B6A1A4311
:2095E0008B6A1A430260CA6842600A6882604968C16070470029016812BF41F001014FF62B
:20960000FE7211400160704704000240080002401C000240300002404400024058000240F1
:209620006C0002408000024004040240080402401C04024030040240440402405804024022
:2096400030B50488DFF8D820DFF8BC30984218BF90420ED0B0F1804F1CBFDFF8B050A8429A
:2096600007D0DFF8AC50A8421CBFDFF8A850A84204D14FF68F752C404D882C43DFF8985035
:20968000A8421CBFDFF89450A84204D04FF6FF452C40CD882C4304808C8884850C88048515
:2096A000984218BF90420AD0DFF8782090421FBFDFF874209042DFF87420904201D1097A5F
:2096C00001860121818230BD0029018812BF41F001014FF6FE72114001807047002A8289C8
:2096E00014BF114322EA0101818170470029018812BF41F080014FF67F7211400180704788
:2097000000BFC94301827047002C01400004004000080040000C004000100040001400405B
:20972000003401400040014000440140004801400300002013F0030F09D0521E22BF13F8B8
:20974000010B11F801CBB0EB0C00F3D07047121F22BF53F8040B51F804CB6045F7D0121DE8
:209760000AD200BA9CFA8CFCB0EB0C0038BF6FF0000088BF01207047521E22BF13F8010BB1
:2097800011F801CBB0EB0C00F6D0521C08BF10467047000000F10103810704D010F8011BD0
:2097A00089B18107FAD10268B2F10131914311F0803F04BF50F8042FF6E710F8011B11B148
:2097C00010F8011BFBE7C01A7047024600E0521C1378002BFBD111F8013B137012F8013BCC
:2097E000002BF8D17047000038B504460D461048FFF742FE05281CBF3420FFF71CFE2946CB
:020000040800F2
:209800002046BDE83440FFF7FDBD10B50446A0050CD10748FFF730FE05281CBF3420FFF7C3
:209820000AFE2046BDE81040FFF7D0BD10BD0000A086010010B5490001F1804101F5C04196
:20984000521C521009E010F8013B10F8014B43EA042321F8023B891C521EF4D110BD49001D
:2098600001F1804101F5C041521C521004E051F8043B20F8023B521EF9D170474FF6F8710E
:209880000840DFF890110860704710B5DFF8882152F8203048F68F142340194324E010B5A1
:2098A000DFF8742152F8203048F6BF742340CC0648BF83F01003890648BF83F020030FE054
:2098C00010B5DFF8542152F820304BF68F742340CC0448BF83F48053890448BF83F40053B7
:2098E00043F4004141F0800142F8201010BDDFF8281151F820204BF68F731A4082F44052C9
:2099000042F4004209E0DFF8101151F8202048F68F631A4042F40042FFE742F0800241F890
:2099200020207047DFF8F01051F8202052040AD551F8202048F68F731A4042F4404242F08E
:20994000800241F820207047334951F8202052060AD551F8202048F68F731A4042F400427E
:2099600042F0C00241F82020704738E0294A126892B202EBC000294A37E03BE02549096849
:2099800089B201EBC00025493AE0224A126892B202EBC000224A2AE01E4A126892B202EBF8
:2099A000C000204A02EB40003F2909D34A091F23194208BF521E1204910941F4004105E0DA
:2099C0004A08C90748BF521C12049109016070471049096889B201EBC000124914E00D4AD1
:2099E000126892B202EBC0000F4A4908490042F8101070470749096889B201EBC0000A49FD
:209A000051F8100080B2704751F810008005800D70470000505C0040005C004008600040B2
:209A2000046000400C600040006000400106090C41EA10207047000080B5964890F820103D
:209A4000022909D018D3042902D00ED3052913D1002180F820100CE0C17B28290CD1816A1B
:209A6000406ABDE8044000F09CBE0121002000F0F3F84FF440512BE101BD38B5854CE57B30
:209A80000220FFF7A5FF60840246D8218248FFF7E6FE94F8200010B1012803D00AE0BDE849
:209AA000314013E02A2D06D1A16A606ABDE8344000F0A1BE022000F0F9F82421052000F07A
:209AC0006BFE00210220BDE83440C5E010B5714C628C1AB170492046FDF77EFB6F486168D5
:209AE0004160A1688160608C1F2806D0022000F0DDF8002020601A218DE0E27B282A18BF1D
:209B00002A2A0FD1607CA17C090441EA0060E17C40EA0120217D08436062A07DE17D41EA87
:209B20000020A06220685E49884270D15D480068617B884204D3A07B401EC0B2102804D345
:209B4000022000F0B3F8242165E0606AA16A002A49D0032A2BD0082A18BF0A2A53D0122AE2
:209B600029D0152A4FD01A2A2DD01B2A27D01D2A49D01E2A23D0232A2DD0252A2FD0282A8C
:209B800035D02A2A37D02F2A39D0552A3BD05A2A1DD0882A18BF8A2A35D08F2A18BF9E2A6E
:209BA00031D0A82A1CBFAA2AAF2A2CD02FE0BDE8104000F0E9BDBDE8104000F0AFBDBDE8BE
:209BC000104000F0EDBDBDE8104000F0D5BDBDE8104000F0D5BDBDE8104000F0AEBDBDE8B8
:209BE000104000F0B9BDBDE8104000F043BEBDE8104000F0D6BDBDE8104000F0FCBDBDE80E
:020000040800F2
:209C0000104000F021BEBDE8104000F038BE022000F04CF82021052000F0BEFD00210120A1
:209C2000BDE8104018E010B50C4622469821FFF701FE21460120FFF7A8FE30210120FFF77E
:209C40002EFE1448032180F8201014488168091B81600021017310BD10B50C460F4B124938
:209C6000196018730D2298211846FFF7E3FD0D210120FFF78AFE0748052180F8201044B1E5
:209C8000042180F8201030210120BDE81040FFF706BE10BD80300020403000202C3100202C
:209CA000555342437C3100205553425380B518B1022807D00AD301BD10210120BDE8044098
:209CC000FFF7EDBD10210120FFF7E9FD4FF480510220BDE80440FFF7F3BD00000278C9B2FC
:209CE0008A421AB11CBF10F8012FF9E718BF002070470000C9B2830706D0521E22D310F8E4
:209D0000013B9942F7D11FE0083A13D302F1040241EA012141EA014150F8043B121F21BFF2
:209D20004B40A3F1013C2CEA030C1CF0803FF3D0C9B2001F083210F8013B521E28BF91EA2A
:209D4000030FF8D818BF0120401E70471B4213D1094236D12AB18446B0FBF2F002FB10C280
:209D6000704700F0E7BDFCD30022002370470B000200002100207047904271EB030CF6D3C2
:209D800070B5B1FA81F4B3FA83F52C1BA340C4F1200532FA05F63343A2405FF00046E6401B
:209DA00002E05B085FEA3202841A71EB030524BF204629467641F4D302000B00300000214B
:209DC00070BD012ACFD970B5140C20D0B1FA81F4B2FA82F5C4F120046419B4F12006D6D341
:209DE000B2405FF00044F440002502E052085FEA3303C61A71EB020E24BF304671466441C9
:209E00006D41F3D302000B002000290070BD0C46B1FBF2F102FB11452D0445EA1045B5FBB2
:209E2000F2F402FB145580B240EA0545B5FBF2F002FB105240EA044070BD30B4436803F022
:209E4000004201211B031B0B436004BF0368002B08D10DE00368DD0F45EA440444605B00CB
:209E60000360491E4468E302F4D523031B0B436043681A434260084630BC70474FF4001CD5
:209E80001CEB410F94BF1CEB430F09E041EA030C50EA4C0C52EA0C0C03D2994208BF90426D
:209EA000704714BF8B428242704700004FF4001C1CEB410F94BF1CEB430F09E041EA030C4B
:209EC00050EA4C0C52EA0C0C03D28B4208BF8242704714BF994290427047000070B5044612
:209EE0000D466068C0F30A5040F2FF72904207D16068000304BF2068002817D0022070BD79
:209F000020B92046FFF799FF012867DA012D0FDB40F2FF71091A8D420AD36068002847BF8B
:209F200000202F4900202F49C4E90001012070BD4142A942616806DA6FF31E51401941EA89
:209F40000050606041E001F000410122636862F31F536360401E451905F13500352803D30C
:209F600061600020206070BD002215F11F0F04DA20352268236000206060684213D0521EE0
:209F80009241D243C0F1200325689D4055EAD2722568C540666806FA03F32B432360636806
:209FA00023FA00F06060606808436060B2F1004F03D80DD12078C0070AD52068401C2060B4
:209FC000206828B96068401C60604FF0FF3070BD6068884204BF20680028F6D1002070BD80
:209FE0000000F0FF0000F07FF446400D40EAC120490006D200F014F8004248BF6FF000406C
:020000040800F2
:20A00000604700F00DF84FF0004188428CBF084640426047400D40EAC120490080F00D80FA
:20A0200040F00040490DA1F58061491C05D4D1F11F0154BFC840C01770474FF00000704724
:20A04000010040F10980F446404200F005F851F000416047010000BF09D0B0FA80F18840F7
:20A06000C91CC1F58461090501EBD0214005704770B44FF0004591EA030F44BF6B4000F0A6
:20A080005BBC00BF841A71EB030604D26E40001BB141121973414FF4001C1CEB410F34BFCE
:20A0A0007CEB430684E00C0DA4EB1356362E7DDC012E43DC45EAC32343EA525312BFD202E4
:20A0C00092025B08240545EAC12141EA5051D2EBC020994125D407D1B0FA80F610FA06F11A
:20A0E00064D00020203608E0B1FA81F6B140C6F1200220FA02F21143B0404FEAF474B4EB50
:20A10000465434F001064FEA74040AD8D6F50016760D04F00044F04061FA06F25040F14007
:20A120004840C00A40EA415021F0004128BF5FEA500550F1000044EBD12137E045EAC323AD
:20A14000DB0A45EAC121C90AB6F120050EDD42EA0242120CC5F1200603FA06F6EB4042EAC5
:20A1600006056D42984161F100010DE062FA06F5F240554063FA06FC82EA0C02F3405A4048
:20A180006D42904161EB030111F4801F05D1641E620502D06D004041494121F48011430851
:20A1A00075F1004350F1000041EB045170BC70471CEB410F15D223F0004352EA43060BD05D
:20A1C0004FEA4C0CBCEB410F04D80C0D661E342EB7DDEBE7801A994150EA410608BF0021D9
:20A1E000E4E708BF1CEB430F28BF6FF00001DDE7B0B581EA030C0CF0004C40F2FF7515EA9D
:20A2000011541DBF15EA1357AC42AF4239E0E41923EA455343F48013C90241F0004141EAC8
:20A22000505EC7021100A7FB020200284FF00000EEFB01204FF00001E3FB072118BF42F030
:20A240000102401800214941E3FB0E01A4F580640F0302D252004041494154F101046CDDB8
:20A26000470872F1004250F1000051EB0451A1F580115CBF41EA0C01B0BD4CEA0551002085
:20A28000B0BD05EA1357AC4214BFAF4241E050EA410E1CBF52EA430E02E061460020B0BD1E
:20A2A00024423C441BD15FEA070EF6D0090302BF01460020AEF1140EB1FA81F7AEEB0704EC
:20A2C00001FA07FE0C37C7F1200100FA07F7C8404EEA000E23EA455343F48013A2E733F001
:20A2E0000043B3FA83F704BFB2FA82FE77440B3FE41BB7F1200E2FBF02FA0EF3BB40C7F18D
:20A30000200E22FA0EFE38BF43EA0E03BA40641C82E750EA410E14BF52EA430E6FF0000186
:20A320004FF4001717EB430F8ABF194617EB410FB5E74CEA05510020B0BDD4F10104B4F151
:20A3400020070FDAC4F12007520828BF42F0010210FA07F501FA07F7E1BF2A43E0403843F4
:20A36000E1400FE0352C98DCC7F1200452EA400220FA07F218BF42F0010231FA07F0A1407C
:20A380000A43002172F1004250F1000051EB0C01B0BD0000F0B540F2FF7581EA030C0CF0F2
:20A3A000004C15EA11541DBF15EA1357AC42AF42E5E0BC41C1F31301C3F31303801A9941FF
:20A3C00043F4801304D2641E4000494180185941C90241EA5051B1FBF3F603FB1611A2FB71
:20A3E0000675D7EBC020A94102D2761E80185941C90241EA5051B1FBF3FE03FB1E11A2FBBE
:020000040800F2
:20A400000E75D7EBC020A94103D2AEF1010E80185941890241EA9051760546EA8E2EB1FBCE
:20A42000F3F603FB1611A2FB0675D7EB8020A94102D2761E80185941C90241EA50514EEA41
:20A44000060EB1FBF3F603FB1611A2FB0675D7EBC020A94102D2761E80185941C90241EAFA
:20A460005051B1FBF3F703FB1711A2FB0735D3EBC020A94167F100070CBF004247F0010773
:20A4800066F3D5274FEA1E31B80814F5806412DDBD0775F1004250EB0E5051EB045111F5A7
:20A4A000801F5CBF41EA0C01F0BD4CF07F6141F0E0410020F0BDBD076D0840EA0E5041F4CC
:20A4C0008011D4F10104B4F120060ADAC4F120060200E04001FA06F3E1401843B2401543BB
:20A4E0000EE0342C13DCC6F1200445EA40056D0820FA06F2154321FA06F0A1400D4300218E
:20A5000075F1004250F1000051EB0C01F0BD00205FEA0C01F0BDCFB992185B41B3FA83F744
:20A5200004BFB2FA82F6BF190B3FB7F120062FBF02FA06F3BB40C7F1200622FA06F638BF79
:20A540003343BA401CB1E419641E33E77F4231F00041B1FA81F404BFB0FA80F6A4190B3CFB
:20A56000B4F120062FBF00FA06F1A140C4F1200620FA06F638BF3143A0403C1B1AE7AC42CE
:20A580001ABF05EA1357AF4212E050EA41061CBF52EA4306BFE750EA4107304661461CBFA5
:20A5A00041EA0551F0BD52EA430C08BFC143F0BD00204FF4001616EB410F98BF16EB430FF6
:20A5C00008BF16EB410F24BFC14305E016EB430F0CBF61464CEA0551F0BD91FBF2F303FB2A
:20A5E0001211C0E90031704770B586B004460D46A68800A8FEF738FE02992948B1FBF0F016
:20A600004FF6C07232400243A28022884FF6FE731A4022802A68234B9A4208D25200B1FBDA
:20A62000F2F18AB2042A38BF042189B220E0EB884BF6FF76B34204D102EB4202B1FBF2F1C3
:20A6400006E019235A43B1FBF2F141F4804189B20A0504BF41F0010189B241F4004189B28A
:20A6600080B24FF4967250434FF47A7290FBF2F0401C2084A183208840F0010020802088E9
:20A680004FF6F5310840A9880843698908432080A88929890843208106B070BD00000000FC
:20A6A00040420F00A18601000029018812BF41F001014FF6FE72114001807047401810F095
:20A6C000030308D0C91A1FD3DB0748BF00F8012D28BF20F8022D130030B414461546103995
:20A6E00028BF20E93C00FAD8490728BF20E90C0048BF40F8042D890028BF20F8022D48BFE2
:20A7000000F8012D30BC7047C91818BF00F8012DCB0728BF00F8012D704700007449087CBB
:20A72000C00702D57348052105E00FF2E410C97C252928BF2421FFF776BA6F480021818002
:20A74000022181710021C1714172022181720021C1720C21FFF767BA6848002101800F21AE
:20A760008170FF21C17000218180022181710021C1710821FFF757BA04216148FFF753BA0C
:20A7800008216048FFF74FBA5948C17C132928BF12215D48FFF747BA5B4A90701173704739
:20A7A00069E070B504460D46584E3078C0B92A462146282000F076F8C8B14D48007B0006BB
:20A7C00003D50220307029460CE00220FFF76EFA00F00EF801210120BDE87040FFF73CBA8A
:20A7E000022804D12046BDE87040FDF7C1BA70BD24210520D0E710B5444C2278EAB90A4600
:020000040800F2
:20A8000001462A2000F04EF8E8B13948007B000608D4012020704FF440510220BDE810405E
:20A82000FFF74EB80020FFF741FAFFF7E1FF00210120BDE81040FFF70FBA012A04BFBDE86C
:20A840001040FDF7E5BA10BD80B52948816829B9007C400702D40121002006E00220FFF7FE
:20A8600025FAFFF7C5FF00210120FFE7BDE80440FFF7F2B900BF01210020FFF7EDB980B57B
:20A880001B48816809B9002004E0007B00064CBF00200220FFF70AFA2021FFF7AAFF0021DD
:20A8A0000120E3E780B55118B1F5805F09D92A2804BF0220FFF7FAF90020FFF7F7F9212140
:20A8C0000BE00B498968B1EB422F0ED02A280CBF02200020FFF7EAF92421FFF78AFF002140
:20A8E0000120FFF7B9F9002002BD012002BD0000803000206831002038040020703100202A
:20A90000600400205404002000040020A030002000800202200000004D696E692044534FF0
:20A920004469736B2020202020202020202020202020202070470000841A71EB030603D2FD
:20A94000001BB141121973414FF4001C1CEB410F34BF7CEB430443E00C0DA4EB1356352E1D
:20A9600050DC45EAC323DB0A45EAC121C912B6F120050DDD63FA05F6EB4086EA03051242C0
:20A9800018BF45F00105C01851F100010CD213E062FA06F5F2405540F3415A40B340F340A7
:20A9A0005A408018594107D349085FEA30005FEA350528BF45F0010501F58011420875F14B
:20A9C000004250F1000041EB045170BC4FF4001C1CEB410F38BF70470020090D09057047E8
:20A9E0001CEB410F10D252EA43060BD0BCEB410F05D80C0DAB43661E342EB5DD02E0AB439B
:20AA00008018594170BC704770BC704710B5DFF8884700B92BE000F096F8006880472068DA
:20AA20000A3010BD80B5DFF870070068C178DFF86C2752788A420CD38278002A04BF82881B
:20AA4000002A06D1817200F07EF840688047002002BD022002BD10B5DFF83C4700B906E0AF
:20AA600000F071F88068804720680C3010BD206801210182002010BD10B5DFF81C4720689C
:20AA8000C1784079DFF8182712689269904721688A7A92B1002804BF087900280DD1887820
:20AAA00058B900F050F8C068804720684179C1722068C1780173002010BD022010BD1CB507
:20AAC000DFF8D416096810B90220088239E0DFF8D44600202080087800227F23184215D181
:20AAE000487A81064CBF42F0020102F0FD0121702178400654BF01F0FE0041F001002070A9
:20AB000000F021F800698047204616BD00F07F03012BF9D000F07F00022812D1487900F02F
:20AB20000F0142F0010200F088FA05D500F030001028E5D12270E3E700F44050B0F5805F12
:20AB4000F7E7002016BDDFF8600600687047F8B5DFF844060068017811F07F0104D1417A08
:20AB600001F0DF0141724FE0022901BF41880029017900294AD1417921F08005DFF82C46EE
:20AB80000A0654F825204CBF02F0300202F44052DFF808361B789D4238D2002A1CBF807ACD
:20ABA000002833D0080654F825000BD500F03000102825D12846FEF7C7FE30212846FEF7E1
:20ABC0006EFE1DE000F44050B0F5805F18D148F280064BF68F7745B900F0BDFA206838406F
:20ABE00080F44050304320600AE02846FEF79AFE54F82500384080F44050304344F82500B8
:020000040800F2
:20AC0000FFF7A1FF406980470020F2BD0220F2BD38B5DFF884050268537923F08000DFF8A1
:20AC20008C151C0651F820404CBF04F0300404F44054DFF868552D78A84206D2558825B933
:20AC4000002C1CBF927A002A01D1022032BD48F280021B0651F8203005D548F6BF742340B0
:20AC600083F0100304E04BF68F74234083F480531A4341F82020FFF766FF80698047002078
:20AC800032BD80B5DFF810050068417A41F020014172FFF758FFC0698047002002BDDFF889
:20ACA000F8241268538A20B98888C01A108200207047086818187047F8B5DFF8DC5428685A
:20ACC00000F110042688A168080018BF002E14D0A088864288BF064630468847074620880A
:20ACE000801B20806088301860800020FEF746FE324601463846FEF7B2FDDFF8B464208838
:20AD000050B1DFF8B0044FF44051018000210020FEF73BFE3020308028682188A2889142AD
:20AD200028BF032101D211B105210172F1BD06210172DFF88404006880B2DFF8801400220C
:20AD400041F8102030203080F1BD2DE9F843DFF84844206800F110063188DFF85454002938
:20AD600004BF007A042816D1DFF85404017801290DD1DFF84414096889B2DFF8402400239A
:20AD800042F8113030212980042703702CE007271020288028E0B6F80480884505D3042784
:20ADA000414588BF4146884600E002274046B168884781460020FEF7E0FD424601464846E4
:20ADC000FEF738FD41460020FEF7DFFD3088A0EB0800308070884044708030202880DFF89B
:20ADE000D4034FF44051018020680772BDE8F18338B5DFF8A4432068457801787F221142B0
:20AE000038D1092D02D1FFF70DFE47E0052D1BD1C17880294FD28178002901BF81880029C3
:20AE2000807A002847D10620DFF88C13096889B2DFF88823002342F81130DFF874133022C0
:20AE40000A802168087231BD032D08D1C178012904BF8088002823D1FFF713FF1EE0012DF0
:20AE600004BFC17801291BD18188C9B9407A80060DD415E001F07F00012804D10B2D0FD199
:20AE8000FFF7FAFD0AE002280AD1012D02D1FFF75EFE03E0032D03D1FFF7BAFE0028C2D034
:20AEA0002846BF49096849698847032808BF0920C7D00028B7D00820C3E738B5B64D286877
:20AEC0004178B74C062913D101787F2211422AD18078012802D12068C16968E0022802D150
:20AEE0002068016A63E003281DD12068416A5EE000293DD14188002904BFC188022912D14F
:20AF0000017981B901787F22114204BF8288002A2CD001F07F02012A10D100F089F810B965
:20AF20002868807A10BB28684078216809698847032845D128680921017231BD01F07F01DD
:20AF40000229F0D1407900F00F0100F0700200F074F84CBF00F0300000F440508F4B1B7872
:20AF60009942E0D2002ADED10028DCD095491EE0082905D100787F210842D4D1924916E0DC
:20AF80000A2902BF017801F07F010129CBD1817A0029C8D04188002901BF01790029C188B3
:20AFA0000129C0D100F044F80028BCD187490800B9D028680022428281610020884700202D
:20AFC00029680A8A4FF6FF739A4208BF092004D0022818BF002A02D10820087231BD0878E7
:20AFE00000061ED5C88800902368009C944202D2009808820FE082420DD293F82C00704C80
:020000040800F2
:20B00000824238BF002005D392FBF0F500FB152008B90120207093F82C008882BDE8314092
:20B0200093E60320087263484FF44051018031BD002140792268926910475C4B000653F85E
:20B040002100704738B55C48006880B2604931F81000400000F1804000F5C0404E4C216802
:20B060000A7A092A14D010F8012B0A70216810F8012B4A70851C35F8040BFEF7D7FC2168E2
:20B0800048802888FEF7D2FC21688880A888C8802068012101722068C08810B9FFF7A8FE1A
:20B0A00001E0FFF70AFFBDE831403EE010B53A4C2068017A022918BF042904D1FFF745FEF1
:20B0C0002068007A14E0062911D14178052902BF01787F22114206D1C07800F042F8FFF725
:20B0E00032FD006A80472E48006880688047082017E010B5284C2068007A022818BF0428DC
:20B100000ED0032818BF052804D1FFF7D5FD2068007A06E0072803D121480068C0688047DA
:20B12000082021680872BDE8104080B500F013F819480068017A082906D11E494FF48052F7
:20B140000A801B4910220A80007A092801D1012002BD002002BD1F4890F82C100020FEF7C9
:20B160001BBC70B50D4909780022104B48F68F760BE0D4B253F824503540254345F40045B1
:20B1800045F0800543F82450521C8A42F1D340F080001149086070BDC83000205C04002011
:20B1A000CC30002084310020D0300020005C00408A31002088310020505C0040046000409E
:20B1C00091310020BFAA00080DAA000857AA000808600040D00200204C5C0040704700001B
:20B1E00080B500F0F8F88B4800680021817200F031F98948002141604FF40441874A118054
:20B20000016087480021016001BD10B5854800218172804800688449C97941720020FEF711
:20B220002DFB4FF400710020FEF72FFB20210020FEF735FB18210020FEF798FB7B4C00F0D5
:20B2400042F858210020FEF790FB0020FEF75BFB0020FEF74CFB00210120FEF716FB9821D3
:20B260000120FEF782FB20210120FEF718FB00210120FEF725FB00210220FEF706FBD82148
:20B280000220FEF773FB94F82C100220FEF784FB4FF440510220FEF713FB00210220FEF79A
:20B2A000FEFA00F010F80020FEF721FB0020FFF758FF5B48012101605D485E4901605E4887
:20B2C0000021017010BD94F82C100020FEF764BB50480068807A00B9704780B550480521B6
:20B2E00001600120FEF730FB0220FEF71BFB52480021017001BD4E4800684E4988421CBF5B
:20B300000220FEF7D3BC704745480421016070477047704780B53F4909680A7802F07F0275
:20B32000212A08BFFE280BD14888002801BF88880028C888012803D10FF28900020001D15E
:20B34000022002BD88610020488200F03BF8002002BD80B52F4909680A7802F07F02212AD9
:20B3600008BFFF2815D14888002804BF888800280FD1C88868B90120FEF7E6FA0220FEF7A8
:20B38000D1FA2B482B4901602B4800210170002002BD022002BD00290CBF002802207047E0
:20B3A0002649FFF77CBC2649FFF779BC19490968C978062901DB00207047224A02EBC10145
:20B3C000FFF76DBC28B91348006801210182002070471D4870471D4801684268806801B9F8
:20B3E000704710B51A4B99700C0A1C710C0C9C71090E19729A72110A1973110C9973110EFE
:020000040800F2
:20B4000019749874010A1975010C9975000E187610BD0000C8300020405C00408E310020A3
:20B4200080310020AC300020A0B80008D00200208030002055534243A03000204404002098
:20B440004C040020000300207C310020E8F7FF1FAC030020064801210160002101604160CC
:20B460004FF4E051034A1180FFE7016000207047405C00408E310020545F5374616E646292
:20B4800079000000545F576F726B0000576169745F54696D6500000049646C655F54696D53
:20B4A00065000000545F5374657000005475726E5F4F66665F76000054656D7053686F77A9
:20B4C000466C6167000000005A65726F505F416400000000545F5374616E6462793D3230D7
:20B4E00030000000545F576F726B3D3330300000576169745F54696D653D3138300000009D
:20B5000049646C655F54696D653D333630000000545F537465703D31300000005475726E53
:20B520005F4F66665F763D313000000054656D7053686F77466C61673D3000005A65726F60
:20B54000505F41643D3233390000000020202023283130307E343030290D0A0020202020AE
:20B56000202023283130307E343030290D0A0000202020232836307E39393939290D0A00AA
:20B5800020202023283330307E39393939290D0A00000000202020202020202328357E32BB
:20B5A00035290D0A000000002020202328397E3132290D0A0000000020202328302C3129D0
:20B5C0000D0A00002020202023526561644F6E6C790D0A002DE9F84F0020ADF8000040F624
:20B5E0008F7848F60F7B48F28006444F444CDFF81491DFF814A14BF6BF7525E054F820109B
:20B60000ADF80010BDF8001009040BD554F8201008EA010144F820103C4901EB800050F8AE
:20B62000040C8047BDF8000000060DD599F8000054F820100BEA010144F82010344901EBBD
:20B64000800050F8040C8047606CAAF80000000452D5BAF8000010F00F0089F80000CDD1D2
:20B6600020683880388800F030007880388800F4405038802068284080F4005080F0200072
:20B6800030432060BAF80000C006206805D40BEA00002060FFF70AFD16E0ADF80000BDF81C
:20B6A0000000000506D5206808EA00002060FFF7C9FC09E0BDF800000004C5D5206808EA3F
:20B6C00000002060FFF715FD206828403988C90448BF80F480503988890448BF80F4005000
:20B6E0007988C90648BF80F010007988890648BF80F0200030432060BDE8F18F88310020DB
:20B70000005C0040923100208C310020E4030020C80300202E48016841F0010101604168BF
:20B720002C4A1140416001682B4A11400160016821F480210160416821F4FE0141604FF4F0
:20B740001F0181600021026842F4803202600268491C920302D4B1F5A06FF8D10168890366
:20B7600030D51E490A6842F010020A600A68920892000A600A6842F002020A6041684160D9
:20B7800041684160416841F480614160416821F47C114160416841F4E8114160016841F001
:20B7A0008071016001688901FCD54168890889004160416841F002014160416801F00C01EA
:20B7C0000829FAD106484FF00061016070470000001002400000FFF8FFFFF6FE00200240CA
:20B7E00008ED00E02DE9F04500F10801026801EB8202406800F001034008400002EB8000C4
:020000040800F2
:20B800000025AA460024A0460126374602E00027F44511D1824201D1BDE8F08552F804CB78
:20B8200003B1CC4452F804EBE644F1E70D686D18091D51F804ABAA445545F7D066B115F97D
:20B84000014B0026012705E00D686D18091D51F804ABAA445545F7D0002C12D50FB115F822
:20B86000018BF445D3D00CF8018B641CF9D40AE0F44518BF5545CBD015F8018B0CF8018B2B
:20B88000641E002CF4D50126C2E70000120100020000004083042057000201020301000005
:20B8A00009022000010100C0320904000002080650040705810240000007050202400000D9
:20B8C000040309042603530054004D006900630072006F0065006C0065006300740072000B
:20B8E0006F006E0069006300730000002603530054004D003300320020004D006100730069
:20B9000073002000530074006F007200610067006500000010035300540020004D00610037
:20B9200073007300FBF7D1F84FF48040FBF705F9FBF7FCF9FBF723FAFBF719F90020FBF767
:20B94000A2F8C820FBF792F80120FBF79CF800F035F8FDF7A0FAFBF751F9FAF747FC0628F9
:20B9600018BFFBF7D0FAFAF752FCFAF715FFFAF733FFFBF776F8F8F7FDFBFBF7EAFDFBF7BB
:20B980003BFEFAF74BFC0020FAF7B2FA40F6B830FAF70EFC084CFAF720FCFAF727FC0628BD
:20B9A00005D0206918B9FBF7FCFA32202061F9F731FFFAF78EFCEEE7D83000200448C06198
:20B9C0000221017203490162034A426208680047AC300020D00200204C03002070B50D4C9F
:20B9E0000D4D286820800D4E208831880840400505D50B48406880474FF6FF302860208834
:20BA000031880840000444BFBDE87040FFF7E2BD70BD00008C310020445C00408E3100206B
:20BA2000D0020020FEF708B8FEF727B810B5074979441831064C7C44163404E0081D0A6899
:20BA4000511888470146A142F8D110BD0800000030000000BBABFFFF302D0000640400206D
:20BA60000000000081FDFFFF0200000002000000A0010000570200000000002064040000C4
:20BA80007047FEE7FEE7FEE7FEE77047704770477047FFF7A3BFFBF7A7B9FBF7C5B9000065
:20BAA00000F009F8002801D0FFF7C0FF0020FFF739FF00F002F80120704700F001B800002E
:20BAC0000746384600F002F8FBE70000C046C046024A11001820ABBEFBE700BF26000200FC
:20BAE000014880470148004715B70008F1BA0008C046C046C046C046FFF7D2FFFFF7C0BFCB
:20BB0000FFF7BFBFFFF7BEBFFFF7BDBFFFF7BCBFFFF7BBBFFFF7BABFFFF7B9BFFFF7B8BFA1
:20BB2000FFF7FEBFFFF7FEBFFFF7FEBFFFF7FEBFFFF7FEBFFFF7FEBFFFF7FEBFFFF7FEBF6D
:20BB4000FFF7FEBFFFF7FEBFFFF7FEBFFFF7FEBFFFF7FEBFFFF7FEBFFFF7FEBFFFF7FEBF4D
:20BB6000FFF7FEBFFFF7FEBFFFF7FEBFFFF7FEBFFFF78FBFFFF7FEBFFFF7FEBFFFF7FEBF9C
:20BB8000FFF7FEBFFFF7FEBFFFF7FEBFFFF7FEBFFFF781BFFFF781BFFFF7FEBFFFF7FEBF07
:20BBA000FFF7FEBFFFF7FEBFFFF7FEBFFFF7FEBFFFF7FEBFFFF7FEBFFFF7FEBFFFF7FEBFED
:20BBC000FFF7FEBFFFF7FEBFFFF7FEBFFFF7FEBFFFF7FEBFFFF7FEBFFFF7FEBFFFF7FEBFCD
:20BBE000FFF7FEBFFFF7FEBFFFF7FEBFFFF7FEBFFFF7FEBFFFF7FEBFFFF7FEBFFFF7FEBFAD
:020000040800F2
:20BC0000FFF7FEBFFFF7FEBFFFF7FEBFFFF7FEBF03040C7480FD000380740C04FC0004034A
:20BC20001C601C03FA000080FC400080FB00011F22FC42012213FC00044040C00080FD4085
:20BC400000C0FD000540407F414040F700016060F600016060F9000078FB04018878FC0086
:20BC6000076050484442414070F000016060F60002E01808FD04020818E0FD00020F302044
:20BC8000FD400220300FFB00020808FCF7000240407FFD4081008100BF006278B4000884ED
:20BCA000B400088CB4000898B40008A4B40008ACB40008B8B40008C8B40008D4B40008E4F8
:20BCC000B40008F0B4000800B5000810B500081CB500082CB500083CB500084CB500085C52
:20BCE000B5000870B5000880B5000894B50008A8B50008B8B50008C4B50008010001E5008A
:20BD000000FADB005780AE80D5805280A8800F80C080D38000804080A0808D801480DA807D
:20BD2000028081803380D980F180DB803080A480A680AF0000E1B100080BB2000811B300DC
:20BD40000813B3000815B3000853B3000897B30008A1B30008A7B30008ADB30008FC0000BB
:20BD600040FD0004C0B8000804FD0004C4B8000826FD0004ECB8000826FD0004AC030020B0
:20BD80001AFD000414B9000810F50003A00FE803FC000033F1000010FD0023DDB10008D15A
:20BDA000B20008DDB10008DDB10008DDB10008F7B20008DDB10008DDB1000809B30008FD69
:20BDC000000201000AEA000010F100018813F60012881300001A03530054004D00330032B6
:20BDE00000310030F3003825BA0008DDB10008DDB10008DDB10008DDB10008DDB10008DD05
:20BE0000B10008DDB1000829BA0008DDB10008DDB10008DDB10008DDB10008DDB10008708A
:20BE2000FA00000AF00011010203040102030406070809020406080001FA0000EFFD0000D0
:20BE400064FA000008FC000002FD00048CB8000812FD0004A0B8000820FC000006FA00049E
:20BE60000301000003FD0000FFFFFFFFFFFFFFFFFFFFFFFFFFFFFFFFFFFFFFFFFFFFFFFFD6
:20BE8000FFFFFFFFFFFFFFFFFFFFFFFFFFFFFFFFFFFFFFFFFFFFFFFFFFFFFFFFFFFFFFFFC2
:20BEA000FFFFFFFFFFFFFFFFFFFFFFFFFFFFFFFFFFFFFFFFFFFFFFFFFFFFFFFFFFFFFFFFA2
:20BEC000FFFFFFFFFFFFFFFFFFFFFFFFFFFFFFFFFFFFFFFFFFFFFFFFFFFFFFFFFFFFFFFF82
:20BEE000FFFFFFFFFFFFFFFFFFFFFFFFFFFFFFFFFFFFFFFFFFFFFFFFFFFFFFFFFFFFFFFF62
:20BF0000FFFFFFFFFFFFFFFFFFFFFFFFFFFFFFFFFFFFFFFFFFFFFFFFFFFFFFFFFFFFFFFF41
:20BF2000FFFFFFFFFFFFFFFFFFFFFFFFFFFFFFFFFFFFFFFFFFFFFFFFFFFFFFFFFFFFFFFF21
:20BF4000FFFFFFFFFFFFFFFFFFFFFFFFFFFFFFFFFFFFFFFFFFFFFFFFFFFFFFFFFFFFFFFF01
:20BF6000FFFFFFFFFFFFFFFFFFFFFFFFFFFFFFFFFFFFFFFFFFFFFFFFFFFFFFFFFFFFFFFFE1
:20BF8000FFFFFFFFFFFFFFFFFFFFFFFFFFFFFFFFFFFFFFFFFFFFFFFFFFFFFFFFFFFFFFFFC1
:20BFA000FFFFFFFFFFFFFFFFFFFFFFFFFFFFFFFFFFFFFFFFFFFFFFFFFFFFFFFFFFFFFFFFA1
:20BFC000FFFFFFFFFFFFFFFFFFFFFFFFFFFFFFFFFFFFFFFFFFFFFFFFFFFFFFFFFFFFFFFF81
:20BFE000FFFFFFFFFFFFFFFFFFFFFFFFFFFFFFFFFFFFFFFFFFFFFFFFFFFFFFFFFFFFFFFF61
:020000040800F2
:20C00000F8FFFFFFFFFF00000000000000000000000000000000000000000000000000002D
:20C02000000000000000000000000000000000000000000000000000000000000000000000
:20C040000000000000000000000000000000000000000000000000000000000000000000E0
:20C060000000000000000000000000000000000000000000000000000000000000000000C0
:20C080000000000000000000000000000000000000000000000000000000000000000000A0
:20C0A000000000000000000000000000000000000000000000000000000000000000000080
:20C0C000000000000000000000000000000000000000000000000000000000000000000060
:20C0E000000000000000000000000000000000000000000000000000000000000000000040
:20C1000000000000000000000000000000000000000000000000000000000000000000001F
:20C120000000000000000000000000000000000000000000000000000000000000000000FF
:20C140000000000000000000000000000000000000000000000000000000000000000000DF
:20C160000000000000000000000000000000000000000000000000000000000000000000BF
:20C1800000000000000000000000000000000000000000000000000000000000000000009F
:20C1A00000000000000000000000000000000000000000000000000000000000000000007F
:20C1C00000000000000000000000000000000000000000000000000000000000000000005F
:20C1E00000000000000000000000000000000000000000000000000000000000000000003F
:20C20000F8FFFFFFFFFF00000000000000000000000000000000000000000000000000002B
:20C220000000000000000000000000000000000000000000000000000000000000000000FE
:20C240000000000000000000000000000000000000000000000000000000000000000000DE
:20C260000000000000000000000000000000000000000000000000000000000000000000BE
:20C2800000000000000000000000000000000000000000000000000000000000000000009E
:20C2A00000000000000000000000000000000000000000000000000000000000000000007E
:20C2C00000000000000000000000000000000000000000000000000000000000000000005E
:20C2E00000000000000000000000000000000000000000000000000000000000000000003E
:20C3000000000000000000000000000000000000000000000000000000000000000000001D
:20C320000000000000000000000000000000000000000000000000000000000000000000FD
:20C340000000000000000000000000000000000000000000000000000000000000000000DD
:20C360000000000000000000000000000000000000000000000000000000000000000000BD
:20C3800000000000000000000000000000000000000000000000000000000000000000009D
:20C3A00000000000000000000000000000000000000000000000000000000000000000007D
:20C3C00000000000000000000000000000000000000000000000000000000000000000005D
:20C3E00000000000000000000000000000000000000000000000000000000000000000003D
:020000040800F2
:20C40000434F4E46494720205458540000000000000000000000188DDD400200D60000008C
:20C420000000000000000000000000000000000000000000000000000000000000000000FC
:20C440000000000000000000000000000000000000000000000000000000000000000000DC
:20C460000000000000000000000000000000000000000000000000000000000000000000BC
:20C4800000000000000000000000000000000000000000000000000000000000000000009C
:20C4A00000000000000000000000000000000000000000000000000000000000000000007C
:20C4C00000000000000000000000000000000000000000000000000000000000000000005C
:20C4E00000000000000000000000000000000000000000000000000000000000000000003C
:20C5000000000000000000000000000000000000000000000000000000000000000000001B
:20C520000000000000000000000000000000000000000000000000000000000000000000FB
:20C540000000000000000000000000000000000000000000000000000000000000000000DB
:20C560000000000000000000000000000000000000000000000000000000000000000000BB
:20C5800000000000000000000000000000000000000000000000000000000000000000009B
:20C5A00000000000000000000000000000000000000000000000000000000000000000007B
:20C5C00000000000000000000000000000000000000000000000000000000000000000005B
:20C5E00000000000000000000000000000000000000000000000000000000000000000003B
:20C60000545F5374616E6462793D32303020202023283130307E343030290D0A545F576FBC
:20C62000726B3D33303020202020202023283130307E343030290D0A576169745F54696D41
:20C64000653D313830202020232836307E39393939290D0A49646C655F54696D653D3336DA
:20C660003020202023283330307E39393939290D0A545F537465703D3130202020202020FD
:20C68000202328357E3235290D0A5475726E5F4F66665F763D31302020202328397E31327A
:20C6A000290D0A54656D7053686F77466C61673D3020202328302C31290D0A5A65726F50D4
:20C6C0005F41643D3233392020202023526561644F6E6C790D0A00000000000000000000A3
:20C6E00000000000000000000000000000000000000000000000000000000000000000003A
:20C70000000000000000000000000000000000000000000000000000000000000000000019
:20C720000000000000000000000000000000000000000000000000000000000000000000F9
:20C740000000000000000000000000000000000000000000000000000000000000000000D9
:020000040800F2
:00000001FF
